:100000004D424E014D3448505001040001000000A3
:100010006000000000C000000000000000000000C0
:100020000000380100000000000000000004000093
:1000300001005001010026000004000000980000AB
:100040000200060127002B00009C000000140000A5
:10005000030006012C002F0000B00000001000007B
:100060000038002035020000000000000000000001
:100070000000000000000000000000000000000080
:100080000000000000000000000000000000000070
:10009000000000000000000000000000550000000B
:1000A0005700000051010000790000008D000000A1
:1000B00000000000FEE708B5044B01221A70044B53
:1000C0000022DA77034B1B68984708BD0000002028
:1000D0000800005034000020034B01225A70A02376
:1000E0000022DB051A70704700000020034B01223C
:1000F0009A70A0230022DB059A7070470000002050
:100100008D23013B002B01D0C046FAE7044B10229F
:100110001B78DBB21807C00F134018437047C04666
:100120002B0000500F4BF7B518261E700E4BA02762
:100130001E70FFF7E5FFFF050B4B01AC00252C37C8
:1001400060701D703E70FFF7DBFF064B20703D7046
:100150001D7023786278181C504040001340034300
:10016000D8B2FEBD2A0000502D00005000230360CD
:1001700030B50B601312012B13D10423013B10D3B4
:10018000084DD4B25D5D641BF8D4074A9D00126827
:10019000AA58002A05D012190260044AD35C1C1B1D
:1001A0000C6030BDE0030000DC030000E40300004D
:1001B00070B58022D2051379DBB2002B19D12B4CFC
:1001C0006360A3602A4B1289261C251C1B6892B20F
:1001D00010361435E260301C291C002B06D09847DD
:1001E0002169002937D1E268301C291CFFF7BEFFC6
:1001F00031E0012B0CD11D4B186900282BD09968D8
:100200005C69A14227DA4C1C9C60137A435422E0BB
:10021000022B1BD1154C2369002B12D06068616939
:1002200088420EDA1B5C1BBAD360124B1B68002B92
:1002300003D0E268101880B29847636801336360A6
:1002400009E080230022DB05DA6004E0032B02D101
:10025000064B00229A60C0468023DB0501221A70FB
:10026000C04602221A7000221A7070BD00000020E1
:100270003C0000203800002080230222DB05FF32F2
:100280001A600421024AFF31118000221A7070475F
:1002900006000040F0B5A023DB059B68534A1F21F0
:1002A0008DB0DBB21160D12B0BD0D02B01D8013334
:1002B000DBB2A022D2059168FF20814319439160EF
:1002C000F1E74B4B4B4A191D043B934203D20022EA
:1002D0001A600B1CF6E7FFF7CFFF474A8023DB02CB
:1002E0001A80464A0027093A92B25A809F80C04637
:1002F000434ADE88434D10685268434C0A922A886C
:1003000009ABB6B21A8123625E810990FFF70AFF3A
:10031000A023DB05DA7C03AB1A7034214D225A701E
:1003200099705A7148214522D9709A7150219C22A6
:100330001971D8716362520005AB0597A3611A80E9
:1003400007AB01220797E3615A70304B0697DA89B1
:100350002F4B08975F882F4B211C1B8828310B706F
:10036000211C1B0A29310B702B4901235B420B70A6
:100370002A482B4903700B702A48211C2E312F3438
:1003800003700B7023702B889E4229D1264B9A4212
:1003900026D0BA4224D1254EF7899F4220D0F68933
:1003A000B446234E7788BC451AD1224FF88998422B
:1003B00016D0FF89EB889F4212D1174B17481A704D
:1003C000120A73880270164A9BB2164813701B0AF1
:1003D0000370EB889BB20B701B0A237000F048F887
:1003E000154B02221A6062B6FEE7C0462800005094
:1003F00004000020400000200004000000C00000B5
:10040000F0BF0000F8BF0000000000200004000062
:10041000FC9B0000FE0300002A0000202B000020AF
:100420002C0000202D000020FFFF0000009C000099
:10043000FCAF000000B0000000E100E01800002068
:100440002030407008080C08FFFFFFFFFFFFFFFF90
:10045000FFFFFFFFFFFFFFFFFFFFFFFFFFFF380171
:100460004D344850434F543200000000000050010A
:10047000F0B5D9B002AF03F0B8FE05F05DFBF8634C
:1004800008F09AFF08F0C8FF09F0F2FB00F078FED0
:10049000CA4ACB4B1A60CB4ACB4B1A60CB4ACC4BE7
:1004A0001A6005F049FB7864052800D142E316D8AC
:1004B000022800D1FFE207D8002827D0012800D168
:1004C000ECE27C6CFC63ECE77D6C032D00D123E354
:1004D000042DF6D105F0B6FB02F0B2FB25E37C6CEF
:1004E000092C00D14EE307D8072C00D136E3082CA5
:1004F000E7D105F0A7FB3BE37D6C0A2D00D153E368
:100500000B2DDED105F09EFB00F0F9FB05F02AFB78
:10051000041E1AD00128D4D1AE4B02221B68391C0C
:100520001D6A7031BD611D691A627D617D6C261C7A
:100530001D61281C3F232A1C8D803D670B7105F02F
:1005400001FCBD637D6C3D64B8E00124012C02D048
:10055000022C0AD098E0002002F06AF803F07CFA3E
:10056000C0B205F03DFC02F049F89A4B6C461B689E
:10057000BC635D681E681B696E43F3189B000A33F9
:10058000DB08DB00E01A8546862502AC6D003C6482
:100590007C19201C0021142209F090F89E204000B4
:1005A0003B1C9021BC333A1849005A607A189A6073
:1005B000391C283A1A61B031143A874D4A60143A0E
:1005C0008A602A688548DC60F03200241470026872
:1005D000386C5361824BB6001B68861910609161BC
:1005E00056602D331A7869465200131C0833DB0815
:1005F000DB00C91A8D4602AB181C211C7B6309F075
:100600005DF805F09FFC3A6C4178331C201C00F02B
:10061000A3FEF86BA04201D005F014FB2B689C6090
:1006200005F0D8FB041C03F017FAA04204D0201CEC
:1006300003F017FA02241DE07C6B3A1C00943B1C6B
:10064000311CBC32B033386C01F062FC624B654A3D
:100650001B68041C9968914202D09A6801329A6022
:10066000002807D105F07EFA002803D105F064FACE
:100670000028D5D0594D00232A6813605360536178
:100680009361BD6BFB63AD4605F06CFA002803D0A7
:10069000002001F0F1F814E705F04EFA002800D12F
:1006A00054E7F5E7022E0DD005F05CFA012800D0E2
:1006B000EDE105F041FA002800D0E8E1012EF1D18A
:1006C00001F09CFF434D6C462B683C6158681C68E8
:1006D0001B694443E3189B000A33DB08DB006946CF
:1006E000C91A8D4602AA7A6302F016FE86200023FC
:1006F00040003A1CFB6564323B185A60043A9A6029
:10070000043ADA60391C043A1A61E431043A4A6066
:10071000043A8A602A686D4690695269A40042438F
:1007200092000A32D208D200AD1AAD4602ADAAB08C
:1007300002A8BD62AAB0F825E85102AAFC20C25165
:10074000264A7D6B12682C191560546053619161C3
:10075000FC6205F0F7FB041C04F074F861780520D6
:100760007A6BFB6A00F0F8FD04F0B4FB1A4BB86A30
:100770001B680024596900F017FCFD6BA54201D0ED
:1007800005F060FA0020391C7831A223021C8C800D
:10079000BC670B7105F0D6FA0F4B1B689C600024F8
:1007A00005F018FBF86303F057F9FD6BA8421BD066
:1007B000281C03F056F9022659E1C046A55D000049
:1007C0003C000020215E000038000020F5100000F1
:1007D00034000020D403002040000020440000200A
:1007E000000E0020FFFFFF7F002C74D1D64B6D461A
:1007F0001B687D6298695A69410001324A43131CA3
:100800000833DB08DB00E91A8D4602AD281C211CE9
:100810003D6308F053FF386CCC4D082808D104F034
:1008200059FB2B68B86A596900F0BEFB3C6450E084
:10083000042003F0F7FA2B68386B5969BA6A05F09F
:10084000D9FF051E012D12D103F0FCFF052003F096
:10085000E9FA391C80318C800C60A323201C221CF7
:100860002C1C00250B7105F06DFA3D6431E0B84D8C
:10087000B86A2B68396B35331A7806F093F82B6811
:10088000B86B35331B785B0098420ADD03F0DAFF62
:10089000052001217A6BFB6A00F05EFD04F01AFB73
:1008A000BC63B96B2B680131B9633433187803F03A
:1008B000D8F803F0EDF82B6800263533187802F0ED
:1008C000C9FE002002F0E8FEF86B03F0CAF803F05E
:1008D00003F97D6AB6E09E4B1B68363318789B4B54
:1008E0001B68186002F0B6FE052003F073FA786BFF
:1008F000F96A00F0E3FE061E06D08621490078184A
:1009000000F0BAFF01249EE06C4692B002AD92B0B6
:10091000FC6002AC8AB0FD6302AD90B03C6302ACF7
:100920008AB07D62311C02AD402288B0F86B3C6217
:10093000FD6108F0C3FE311C4022386B08F0BEFE9A
:10094000311C2022786A08F0B9FE311C4022386A36
:1009500008F0B4FE02AC311C2022F86908F0AEFEAB
:10096000201C311C202208F0A9FE902040003D18D8
:10097000F96B3A6B7B6AAC61764C6960AA60EB609C
:10098000386A2368F9698622520028616961281C47
:10099000B9181D63102200F0CBFE9E204000391CC8
:1009A0003C18BC3161600C39A1604439E160043904
:1009B00021613B1C6749D03363611E605E603A1C55
:1009C0000B684C32A2611C6186235B001680FA180A
:1009D0003B1CE433281C211CFE66BE6600F0DEFED4
:1009E0006068A16806F010FA6068A1680230023100
:1009F00006F00AFA381CF830396C07F09FFE3864AC
:100A0000032804D0072800D07FE1182505E0381C12
:100A1000F83008F0EFF9051E09D005F0B1F86B1EAB
:100A200001229A401040D84000D16EE184E103F0E9
:100A3000C5F903F08FF80124464B00221B681A61A8
:100A40001A63FD68AD46414B434A1B689968914261
:100A500002D09A6801329A60002E08D105F082F81F
:100A6000012804D105F068F8002800D198E603F0C9
:100A7000A5F903F0E7FE374B1A68002313605360B3
:100A80001361536193613C69FB63A5460CE62E4BF1
:100A9000BD691B687C691D621C6112E505F0D2F816
:100AA00005F04AF80128FBD008F062FC00F068FB72
:100AB00004F046FE05E500F0B3FE264B1B685869BE
:100AC00000F0DAFE04F07EFF05F0BCF805F0D4F883
:100AD000032812D006D801280CD0022815D102F024
:100AE00011FA12E005280ED00AD306280DD102F023
:100AF00083FD0AE002F0C0F807E002F0A3FA04E088
:100B000004F048FC01E002F065FD05F015F802284C
:100B1000DCD000F097FED4E405F094F801F06EFD0F
:100B200005F00AF80328FBD0CBE405F005F804280B
:100B3000FBD0C6E405F086F803F08CFB04F0FCFF64
:100B40000528FBD0BDE4C046D403002040000020AF
:100B5000000E002044000020FFFFFF7F05F072F828
:100B6000012001F065FD04F0E7FF0728FBD0A8E4B1
:100B7000002003F057F903F039FA04F0DDFF0828EC
:100B8000F6D09EE405F05EF8002002F02EFC002076
:100B900003F048F903F02AFA04F0CEFF0928F6D052
:100BA000012002F022FC8CE46C4600207C6308F0FB
:100BB00069FC08F031FC002003F00AFA6D4D2B6847
:100BC0005E6818681B694643F3180733DB08DB00CF
:100BD000E11A8D4602ACA619FC6202F07FFB02F01E
:100BE00095FB02F087FBF86A311CFE6303F0E4FB1F
:100BF0002B686D465A681B69D3189B000A33DB08C3
:100C0000DB00ED1AAD4602AC3C6405F01BF8594D13
:100C1000391C2B68983118681A7908704A708A70E4
:100C20005A1DD27F1B69FC6ACA700B710022012316
:100C30004B710420131C009405F04AF8F96BF86A14
:100C400004F0C8FA002003F0EDF82B684A495D680B
:100C50000E68BD630022B86B824208DA90008446B9
:100C6000B069644600593D6C01322851F3E73C6C91
:100C70008200A4181D690E68A4460022AA4206DA62
:100C8000306A91004058644660500132F6E7BA6B12
:100C9000391CA03118684A709A6808708A70053348
:100CA000DB7F0132CB70344B92001B680D715B69A6
:100CB00004259A184D7100920022131C022005F0A1
:100CC00007F8391CA83101230B702A4B3C6C1B68B8
:100CD00005201A794A708A705A1DD27F1B69CA7022
:100CE00000220B714D71131C009404F0F1FF04F00D
:100CF00023FF0A288BD07D6BAD46FFF7E2FB04F0A3
:100D00001BFF0B28FBD0FFF7DCFB3C6C082C00D052
:100D10008DE603F053F8012002F091FC0024391C09
:100D20008831A223201C221C8C800C600B7105F0E2
:100D300009F804F0CFF87FE602214820C155381C9D
:100D400049224830D55504F083FE03F037F80120DE
:100D500002F075FC0024391C9031A223201C221CB7
:100D600008258C800C600B7104F0ECFF04F0B2F8E5
:100D70003D6461E6D403002040000020F8B5184D22
:100D80007146281C764603F07BFB164C276802F060
:100D9000F7FE7862276802F0F7FEB862276802F073
:100DA000F7FE7861276802F0F7FEF861276802F025
:100DB00045FFB861276802F057FF0B4B0B491B68D2
:100DC000096838621878097C22684143023311614E
:100DD000E832281C311C136003F06AFBF8BDC046E2
:100DE0001D0D000040000020040E0020000E002019
:100DF000014B18607047C046000E0020014B186878
:100E00007047C046000E0020014B18607047C04676
:100E1000040E0020014B18687047C046040E0020E5
:100E2000014B18687047C04640000020014B5868CD
:100E30007047C0464000002082B0F0B589B0109CD9
:100E4000151C0F930693029407900E1C119C02F040
:100E500045FA47793A4B04978279964206D11B6846
:100E60000021DA69AB00D05A03910BE01A68354BC8
:100E700052691968731C896803964B43EB18013358
:100E80009B00D05A0499714349194A00A418238839
:100E9000069E0193019F7318874203D8C61B029FC9
:100EA000BE521CE0029EB61805960027F65F01367A
:100EB00010D01F787EB2B446013601DA013703E064
:100EC0006646002E06DD013F1F7002235B42238031
:100ED00001202FE0069F79180F78002F01D1208084
:100EE0000CE07FB27C1C05D1019E059F301A388032
:100EF000002002E0012F01D1FF2008701978039C27
:100F0000049E079F48B274437D19002805DC029EA9
:100F1000B25E013208D0002906D12A5700203E2AAD
:100F200008DC0131197005E02A57002A01DD01397A
:100F30001970002009B0F0BC08BC02B01847C046C8
:100F400040000020D403002070B5154C7146201CD1
:100F5000754603F095FA134B00221B68191C883163
:100F60000A601E1C01219C364942181C3160B26087
:100F70000830083EF18232607283C26790300160AF
:100F8000826008380183191CAC31026004330A8086
:100F900020390A60201C291CDA6703F089FA70BD29
:100FA000E90E000040000020F0B5754685B00395BD
:100FB000294D01900F1C281C714603F061FA274B44
:100FC00000211B680198DA69920008F077FB04F0B1
:100FD000B9FF02904478214D002C21D0042002F06A
:100FE00021FF28684269561E009617D3836900992D
:100FF000019E5943C918890071180439013B0BD36C
:10100000866856439E190136B600F5590E68AC46FF
:10101000B44465460D60F0E7009AE4E7013CDAE786
:101020002F687D69013D11D3BC69019A261C6E436E
:101030003619B6009619043E013CF3D3029B306882
:10104000597808F02BFA00043060F4E7024803995D
:1010500003F02EFA05B0F0BD490F0000D4030020C4
:1010600038B50B4C7146201C754603F009FA094B44
:10107000201C1B68DA6A002A03DD596B5218D20F54
:1010800000E000227433291C1A7003F011FA38BDF5
:101090000110000040000020F0B52C4F72468BB0CC
:1010A0007146381C019203F0EBF9294D2B681A1C8C
:1010B000CC321178583A002904D1191CB031097882
:1010C000002901D0002111701478002C21D0996FD3
:1010D000002407915A6B03A90892DB6A07AA0993B7
:1010E00003234B708B707C235B42CB700126102353
:1010F000201C8C800E700B7104F024FE2B689A6FFC
:10110000D96F8A4202DC92199A6718E09C67341CF6
:1011100015E05A6B05A90792DB6A092008930123A1
:101120000B7002234B708B707C235B42CB7007AA41
:1011300064238C800B7104F005FE2B689C67381CBF
:10114000019903F0B5F9201C0BB0F0BD3910000077
:101150004000002038B5094C7146201C754603F04C
:101160008FF904F0FFFC002802D1022002F032FEC9
:10117000291C201C03F09CF938BDC046F510000066
:1011800037B5114C7146201C754603F079F905F00E
:1011900083FC02F0BBFE021E07D16946A9238880AA
:1011A00000900B7104F0CEFDFEE7084B1B6803CBEB
:1011B00002F028F905F088FCFFF7E0FD291C201C4F
:1011C00003F076F937BDC04621110000D40300209A
:1011D000F0B587B000AF7546786039615C487146FC
:1011E000FD6003F04DF903F091F883000A33DB084A
:1011F000DB006E46F61AB546041C684603F08EF80E
:1012000063000833DB08DB00F61A301C6D46B54678
:10121000BE6003F09FF84F4B1B68191C88310868AB
:10122000632807DD0120002240420A604861CA614C
:10123000191DCA671A1C88321068191C0130083140
:101240001060CA6F632A09DD00220120CA6740428C
:1012500090318A6008601A1D0121D1671A1C08327A
:10126000D16F0131D167191C94310E68012E07DD51
:101270000120002240420A60C8824A8308390A607D
:101280001A1C9432116801311160191C90310868E0
:10129000012809DD002201200A608A8340421A1CCD
:1012A00008838C32012111601A1C903211680131BF
:1012B00011600022101C013C08D3A1006958BE68CF
:1012C00040186100715A521892B2F4E7191CAA3101
:1012D0000024A4261D19B446AC447D6165462D68E2
:1012E000854201D2664630607E699C36356885420B
:1012F00000D930608E88964200D28A800E8896424D
:1013000000D90A80043C261C02390836E1D11A1D96
:10131000D26F7D6892009A18111CA031983209682A
:1013200012683E698A1A2A801A1C8C321268084890
:1013300052009B181A1CAC32A83312881B88F9681B
:10134000D31A338003F0B4F8BD4607B0F0BDC046F1
:101350007111000040000020F0B5284E85B07546A0
:101360000191041C7146301C1F1C0395009203F070
:1013700087F8234D00212B680098DA68920008F066
:101380009DF92B68381C1A690021920008F096F923
:10139000019D002D0CD0201C02F044FD194B00983B
:1013A0001B68391C5A69DB6905F0EAF9013DF0E771
:1013B000002C0FD1134B1B685D699E69029502F0EA
:1013C000CEFB051C02F0D4FB311C031C2A1C029826
:1013D00004F0D0FD0098391C019A04F033FF002C72
:1013E00006D1084B201C1D6802F0D0FEEC352860A9
:1013F0000248039903F05CF805B0F0BDF912000053
:10140000D403002040000020F0B595B004AF75462D
:1014100078613961A3487146FA61BB61FD6003F0F0
:101420002FF804F08FFDA04B6C461B68BC601C6855
:10143000786204346400221C0832D2086846D20064
:10144000851A5A68AD4604325200131C0833DB0873
:10145000DB006846C01A04AD854604AE301C00218E
:101460003D6208F02BF9221C0021386A08F026F9A9
:101470008E4C7D6923685A69191C9B690095386AEE
:101480002C3104300190301D0290F86904F07CFF8B
:101490002368874D191C68313960796A78602A6839
:1014A000097B586992680091396A029601912C3340
:1014B000396807F017FDBA68236838699546191C22
:1014C000DA691B6A00902C31B86905F0BDF87E68B6
:1014D0000643F6B23E6204F047FD0679012E0BD1B9
:1014E0002B685B691B78002B06D104F03BFB0128BD
:1014F00002D0301C02F0A3F82568281C291C683192
:101500002C3004F007FF6B4A23681268E8660C244D
:10151000115F9D6D8D420EDC0E20115EDC6D8C42E4
:1015200009DB1025515F186E884204DC1221525EDF
:101530005B6E934221DA00233B8738220123D35587
:1015400004F02CFB002818D104F08CF9002814D0EA
:10155000564B1A68FF239168FE2901DC9368DBB2C1
:10156000381C022139243830E35504F071FA52480E
:1015700002F0DAFF01F064FFE2E74B4E2921336805
:1015800028255A681868CA559A682A23DA5580238C
:10159000E8555B4202252B432B200024C3552C2108
:1015A0005323BC850132CB55FB695200391C9A1874
:1015B0000120283104F0C6FB32680121137C302061
:1015C000C15531203221C355CB5580235B422B437B
:1015D0003322D35534206D23391CBC863031C3559A
:1015E000BA69012004F0AEFB336838211A6839204B
:1015F000CA555968C1559A683A20C255591DC97FC4
:101600003B20C1551B693D203C21CB55C35D7F214B
:101610008B43802149422B430B430132F96952002D
:101620008A18391CC35538310120231C0092221C12
:1016300004F04EFBFFF714FDFFF72EFDA04227D16B
:101640001A4C2368586902F01BFD2368D86E02F01B
:1016500011FC02F0DDF93D6A002D0DD12368F96916
:101660001A1C2C321B68786904F000FD2368386965
:101670001A68B96904F056FD022002F00DF8B86945
:1016800005F0EEFA20680024703006F04BFE00E012
:101690002C1C0448F96802F00BFF201CBD4611B059
:1016A000F0BDC046A9130000D40300204000002074
:1016B00044000020040E002010270000F7B5194C4C
:1016C00000AF73467960061C7146201C3B6002F037
:1016D000D7FE154B68461B68144D19689B688A1C19
:1016E0005B005A4301315B084B430832D208D200F9
:1016F000801A8546013329686A465B00D3188A60E0
:10170000CB60301C7968FFF77FFE2B680022061C37
:101710003968201C9A60DA6002F0CAFEBD46301CAF
:10172000FEBDC0465D160000D4030020440000202A
:10173000F0B585B002AF7446051C3C607960141C9E
:101740007146144802F09CFEA200131C0A33DB0809
:10175000DB006946C91A8D4602AC201C002107F047
:10176000ADFF0D4E281C3268516A936A68320092B0
:10177000221C06F0F9FD33687A68596A281C9B6AB6
:101780000092221C06F05AF93968024802F090FED5
:10179000BD46F7BDD116000040000020F7B51E4F32
:1017A00075460C1C161C7146019500901D1C381CBA
:1017B00002F066FE211C2B1C321C009806F06EFB0A
:1017C000201C05F0ABFC154B201C1B68596A9A6A5B
:1017D00006F07AFC201C05F0D7FB2A1C201C311CCB
:1017E00005F06CFA04F0C0FB051C05F067F99E30AB
:1017F00003783C1C002B09D12B79002B06D004F078
:10180000B1F9012802D0012001F019FF201C019933
:1018100002F04EFEF7BDC0463D170000400000201C
:1018200038B5074C7146201C754602F029FE07F0BA
:101830006FFD01F059FD291C201C02F039FE38BD56
:10184000C117000038B50B4C7146201C754602F0DC
:1018500017FE07F01DFE07F063FD01F045FD0020B7
:1018600002F0B6FB01F0C8FE291C201C02F020FE8D
:1018700038BDC046E5170000F0B5C5B000AF7346EF
:101880007146041C38487B603E1C02F0F9FD381C90
:101890002C360021142240303D1C07F00FFFE835A4
:1018A000301C0021142207F009FF00212822281CE7
:1018B00007F004FF381C0A220C30002107F0FEFE5E
:1018C0003B1C6833D022D351143BD422D351402344
:1018D000DB19D822D351DC23DE51E0220C23D55171
:1018E000DB19E422D351204E002C2AD16A46583D00
:1018F0003A60281C211C142207F0E0FE3B1CB83380
:10190000FB61143B3B62283BBB62184B7D621B684A
:101910001B6A5B00023B9A1C02D0FF22EA52F9E7E5
:10192000381C391CCC30183105F012FA05F042FA97
:10193000381C391CCC30183105F0B0FC3B689D4692
:101940000BE0381CCC30211C05F002FA05F032FA0D
:10195000381CCC30211C05F0A1FC301C796802F049
:10196000A7FDBD4645B0F0BD19180000D403002006
:10197000F7B5304E7146301C754602F081FD05F01A
:101980009DF82D4C9E30236801781A79002902D1E8
:1019900051B2481C04D10027DF60BA420DD118E0D3
:1019A000D8681A69904202DAD8680130D8600129F3
:1019B0000FD0DB6893420CDB012700223B1C6946F9
:1019C0000E33101C8A8000920B7104F0BBF923685F
:1019D0001F7123681A79002A03D1184A12681278F5
:1019E00004E0012A03D1154A126852781A60186877
:1019F00002F076FD2368071CEC33186802F094FDB2
:101A00003F1A002F0BDD2368186802F069FD236878
:101A1000071CEC33186802F087FD381A00E001203B
:101A200001F00DFE01F02CFE301C291C02F040FDDF
:101A3000F7BDC0461119000040000020040E002030
:101A4000F0B5734691B0041C0E1CAF487146059367
:101A500002F016FD04F088FA049005F02FF82278C1
:101A6000AA4B002A08D17A300278511E8A41D2B29C
:101A70000292002A06D001E0012002901A6800219B
:101A8000B83205E01A68B8321168FE2901DC01316C
:101A900011601B6800211A1CB432117002990029D0
:101AA00004D09B490968097D00295FD0181CB33018
:101AB0000178C9B2002908D003785BB2022B00D0AC
:101AC000012313700023037084E11D1CB0352C78B2
:101AD000002C09D0012414701A1CB132BC330170DF
:101AE00029701170196076E1029800283ED1191C06
:101AF000BC310C68002C09DD013C012C01D00C60CC
:101B000034E0029B0B600323137064E11A1CE8327B
:101B1000126811887F4A914228D01A1CC832118855
:101B20007D4A126852888A4220D8794C2068427CCB
:101B3000181CB8300068904218DB0EAA1180CA3316
:101B40001B8806A95380029B02988B8001230B708F
:101B500002234B708B70CB7015230B7104F0F2F8DD
:101B60006A4B22681B68927CBC331A60684C2768F9
:101B7000F87C002800D02DE10299644D002900D0A6
:101B80008AE02C68231CE7331B78002B5CD03B1CBD
:101B90002C331B78002B57D0231C0E91DC331B6891
:101BA0000393231CC83303981A8843009A533B1CA1
:101BB0002D33197802984B00F618031C994206D071
:101BC0005A00B21A023A128801338018F6E707F079
:101BD000B3FC0E90FA8B231CE033904202DA1A68B1
:101BE000013200E000221A603B1C221C2E33E0323E
:101BF0001B7812689A4219DD7C2308A900265B42F3
:101C00000124CB70301C16230EAA8E800C700B7131
:101C10004C708C7004F096F82B68301C1A1CDC3267
:101C2000E03316601E6004F0CFF8D4E03B1C2D3387
:101C30001A780399231C013ADC33914202DA0A1C18
:101C4000013200E000221A60C4340137FB7F2268B1
:101C50009A4219DB00240AA91223201C221C8C8022
:101C60000A940B7104F06EF82A682948131CC033DB
:101C700019680068013119600230C07F814203DBBE
:101C80001C60B432022313702A680023111CB23185
:101C9000C4320B70136049E02B681A1CBC32106010
:101CA0002A321278002A41D0191CC83109880EAA9C
:101CB0001180CA331B880CA9538001230B700223A7
:101CC0004B708B70CB70192388800B7104F03AF83D
:101CD0002B682268191CC8310C88D08B16398442B5
:101CE0001CD2181CCA300488508D844216D2097840
:101CF00000291BD1C43301321968D27F914215DA11
:101D00000131196012E0C046E119000040000020D6
:101D1000000E0020FFFF0000040E002001220A70C8
:101D2000191C0022C431C0330A601A602D4D2B6883
:101D30001A1CE6321278002A4CD104980279002A43
:101D400046D01A1CB0321478002C43D1264ED86AE3
:101D50003768798BBA8BFB8A3F8B009704F0ACF81D
:101D600036682B68718CB28C071CD86AF38C368D60
:101D7000009604F0A1F82B681A1CC8321188CA33E7
:101D8000B94202DA1A88824214DB08AA11801B8841
:101D90000EA953800223002001254B708B70CB705D
:101DA000172388800D700B7103F0CCFF0D4B1B685F
:101DB000B1331D700B4B1B681A1CB1321278002A0C
:101DC00008D00299002905D0B03301221A7002E030
:101DD000B1331A7001240548059902F069FB201CF3
:101DE00011B0F0BD40000020000E0020E1190000FD
:101DF000F7B575460195424D7146041C281C02F04A
:101E00003FFB404E33681A1CB1321278002A24D0AE
:101E10001A1CE6321278002A1FD11A1CCC32117813
:101E200000291AD1B0331B78002B16D1012313706F
:101E300001F060FA071C01F051FA334A031C1268E2
:101E40005D3303CA3A1C9B3204F0AEF901F0B6FFD1
:101E5000022001F0BFFFFFF777F833681A1CCC327D
:101E60001278002A45D01A1C0020B0321070274A80
:101E700000901768011C3A6A013A0BD3E5685600D6
:101E8000755B002DF8D02EB20131B042F4DA301C6F
:101E90000092F1E71A1CE6321278002A0ED10129CD
:101EA0000CDD012222703A6A013A09D300998A4274
:101EB000FAD0E568510000204853F5E7002903D027
:101EC0001A1C0021D43208E01A1C181CD432D0305D
:101ED00011680068814201DC013111601A1CD432A2
:101EE0001168043A1268914205DDB03301221A707C
:101EF00001E0D4331A600248019902F0D9FAF7BD23
:101F0000911D00004000002044000020D403002068
:101F1000F0B5C1B002AF7546F861B961D9487146F4
:101F20007D603A62BB6002F0ABFAD74E6C46326815
:101F30003C61136892689D1C520055430133291C73
:101F4000520853430831C908C900601A8546013355
:101F500002AC5B00FC62E318CC4CBB622368FC6AF9
:101F600000219C60BC6A3C22DC60C94C20682C309B
:101F700007F0A4FB2A1C0021F86A07F09FFBA623A8
:101F80000020382100253887CB55391C2A1C281CF5
:101F900034317D6303F0D6FEFFF7EAFC21683C256F
:101FA000081CC830CA31FFF713F9316800234022FA
:101FB000D35301200B79E8553D223E25D355EB55EF
:101FC00040225B23D355042123683F20C155391C8F
:101FD0009A6902203C3103F0B5FE3268002548239F
:101FE000DD530121137C4420C15545254620EB5586
:101FF000C35548256C23EB55042223684721CA5555
:10200000391C1A6A0220443103F09CFE23683D1CEF
:102010001A1CC8321288DC352A80CA331B88391C46
:102020004C310122002088800A700A716B800C20DC
:1020300002232A1C4B708B70CB7003F083FE336835
:10204000391C5A68186854314A709A680870581DCB
:102050001B698A70C07F0B7104234B7123680132A6
:102060005B6992009A18C87000920022131C02202B
:1020700003F02EFEF869B969FA6ABB6AFFF7C4F982
:10208000F862002803D0386AFFF7F6FBCEE0684616
:1020900092B002AC92B0BC6202AC8AB0FC6102ACFD
:1020A00090B002AE8AB0BC6102AC88B0F8607C62CD
:1020B000F96A02AC4022B86A7C6107F0FFFAF96A5B
:1020C0004022F86907F0FAFAF96A2022B86907F0A5
:1020D000F5FA301CF96A402207F0F0FAF96A20227A
:1020E000786A07F0EBFAF96A2022786907F0E6FAD5
:1020F0003C1CF969C034B86A7B6AA1606349BA695B
:102100006060636178690B68E2601C63A061396A92
:10211000201C10222661FFF70BFB3E1C8AB002AA8E
:102120008436BA62F96A1422301C07F0C7FA381CE8
:10213000F96A1422703007F0C1FAF96A2822B86AE5
:1021400007F0BCFA381CF96A0A22643007F0B6FAC4
:102150003B1CAC336B60143BAB604C4A7023DB1907
:102160002B61B86A13686421C9196861A961EE60BE
:10217000201C1D61291C3A6ABB68FFF70FFB8823EE
:102180005B00D959281CFFF75BFC424B1B681B7D89
:10219000002B02D1281CFFF72BFE3C1CDC34201C3A
:1021A000396A05F07BF825786C46AB000733DB080D
:1021B000DB00E41AA54602AC3C622E1C12243B1C38
:1021C000DC33D868025F002A09DD3A6A013E5B69A8
:1021D000B000610010185918042207F02DFA023CD3
:1021E000A31CECD1284B391C1B685C311C68586857
:1021F0009A680C7048708A700533DB7F0132CB70AF
:102200007E235B424B71224B52001B6800249B6A69
:102210000C719A1800923B6A03202A1C03F058FDA7
:102220001A4B1B681C611C63FC68A546174B0022F7
:102230001B689A60DA603D69AD4601F08BFC01F0E5
:10224000BDFD01F053FA012001F0ECFD01F0A2FB0D
:102250000F4BB4201B68185600F0F2FB041E00D18F
:10226000FC6A0D4B1B681A680C4B9A4202D001F0B5
:10227000F1FFFEE70348796802F01AF9201CBD4619
:102280003FB0F0BDB11E0000D40300204400002088
:1022900040000020000E0020280E0020CDCDCDCD26
:1022A000F0B59DB002AF74467146CF487C6002F035
:1022B000E7F801F013F8061C01F028F8386101F086
:1022C00019F8CA4B6D461C68B860E36800211A1CF7
:1022D0000E32D208D200AD1A2269AD460E32D208B3
:1022E000D2006846801A02AD8546FD6102AD7D626E
:1022F00072799A18131C0E33DB08DB00C01A5300E6
:102300000E33DB08DB008546C01A02AD8546C01AD5
:10231000BD6102AD854602A87861B86907F0CEF9C3
:10232000E1687279281C521801215200494207F0D5
:10233000C5F9E3687279AE49D2185200786907F09E
:10234000BDF9E2683969F8693D6607F075F93D69DC
:10235000F020800029182269786A4024002507F0BF
:102360006BF9FC603D62796AF86902F033FF032083
:1023700001F058FD9D4D00202B6838861A6858687A
:102380002C212D24CA55E0559A6804242F23DC55AE
:10239000984C51233020C35523682E21CA555B69C0
:1023A00001329200391C9A1802202C3103F0CAFC29
:1023B00001233422D3552B6836201B7C3525EB5561
:1023C000C35500215A233825398704223721EB557C
:1023D0002368CA55391CDA690220343103F0B2FC93
:1023E000B479013C631C2CD07579013D6A1CF8D08E
:1023F000737978696343EB185B001A5A7E4B9A42F3
:10240000F3D0B96960223960F9657866D2196946F6
:1024100009CA09C1211C3B68F8692A1CFEF70CFD9A
:10242000002803D03B6A01339BB23B627379BA69DF
:1024300063433869EB18D15CC25C8A18F969CA54E5
:10244000D3E7F479013C601C30D0B17973797D69B0
:102450004B43E3185B005A5B674B9A42F2D0BD696D
:1024600060203D60FD65C0197D6984467D666846D3
:10247000624628CA28C0221C3B68786AFEF7DCFC4A
:10248000002803D03B6A01339BB23B627379B27977
:10249000BD695A432B193D69F0202919800009189C
:1024A0009A5C0B787D6AD3182B55CBE74F4B3C6A6F
:1024B0001B68DA681B69D3189C4206DAFB68013B8B
:1024C000DBB2FB60002B00D04DE700244025FC630D
:1024D000EC53B3793C20C35573793D213E223F250F
:1024E000D355CB55EB5D7F200125834380212B43C2
:1024F00049420B433F22D3554020D223391CC355B8
:102500003C310820FA6903F01DFC391C44317C641D
:102510008C800D70F3797F224B708B70CB78082004
:1025200093431D4380235B422B43CB707A6AD323B2
:102530000B7103F007FCB379013B0FD37279013AB9
:10254000FAD37179BD685943FC698918E818611894
:10255000A4300C78007820180870F0E7F379013B7C
:1025600008D3BC687D6AE218C8321178EA5C8A1820
:10257000EA54F4E7F869796A02F02CFE391C4C3110
:102580000024FC648C80B3797F200B707379012563
:102590004B708B70CB78802283432B435242134382
:1025A000CB70FA691D2308200B7103F0CBFB391C9B
:1025B00054317C658C800D70F3797F244B708B7067
:1025C000CB788026A3431D4376421E237A6A2E438E
:1025D00008200B71CE7003F0B5FB0348796801F059
:1025E00067FFBD461BB0F0BD41220000D4030020B0
:1025F000FFFF000040000020FEFF000038B50B4C3C
:102600007146201C754601F03BFF00F073FE9830C8
:102610000378002B02D1FFF743FE01E001F0FEFE3C
:10262000291C201C01F044FF38BDC0469D25000038
:10263000F0B5A5B000AF724671467861E1487A60A6
:1026400001F01EFFE04C23689B683B625B00013396
:102650003B6501F0F1F92368FF229B68F865D31A06
:10266000984200DDFB65F86D3B6A0024C31AFB61EC
:1026700001F0EAF93A6D694655002B1C0833DB0876
:10268000DB00C81A85466A466423DC5360200123B8
:102690007965FA6461216222C355CB55D3557C23F9
:1026A0005B426320C3556421B123CB553A1C391CCE
:1026B000201C60315C3203F045FB3A6D944206DA2F
:1026C000F869F96C63002218CA520134F5E7002456
:1026D0006C23D1B2DC530126682069226A23C655D7
:1026E000D155D955B96402236B20391CC3556831C3
:1026F000201CFA6C03F026FB2B1C796D08338D46E9
:10270000DB08DB006A46D21A9546D21A694695461E
:10271000F9637A6301F0FAFD3861301C01F01EF8AC
:10272000211C2A1C786B06F0C9FF211CF86B2A1C9F
:1027300006F0C4FF386D69468000031C0A33DB08CD
:10274000DB00C91A8D46C91A3B69B8619B0068460F
:1027500038638D46F962BB60FC640021BA69386B4E
:1027600006F0ACFFF86AFF21BA6906F0A7FF002067
:102770007865954B786D1B685B6898424BDAF96910
:102780000026C9B2081CB96301F06BF901F034F9F5
:1027900000F0DAFFFC6A3D6B386D0136F217C30FAB
:1027A00086425341DBB2BB62002B06D1B96B88195C
:1027B000C0B201F056F901F01FF96B46FB60BB682F
:1027C0006A460A33DB08DB00D01A85466A467A641B
:1027D00001F0A4FD00231A1C39698A4205DA786CDD
:1027E0009100415801325B18F6E72A68934200D9FC
:1027F0002B602068834200D22360F968BA6A8D4654
:1028000004340435002A02D100F09EFFC4E77B6D3A
:1028100001337B65ADE700216C4D79650C1C3A6D89
:10282000944217DA3A6BF96AA300D058CB58C01A11
:10283000854204DDFA69051CA2187A623C647B6D4E
:10284000834200DA786500F073FFF96B6300C852C9
:102850000134E4E7786D00F06BFF5B4B1B685B882D
:10286000984206DA7B69012B03D0F86D396A7862E9
:102870003964574D00262C683222231DDE6704334D
:10288000DA67396C803364221A60022291409A60C0
:10289000FA6A01208A58D8605E60101C3A60B963F9
:1028A00000F046FF9834BB6B396B206058582C6899
:1028B00000F03EFF2B6801211A1CAA32A0344942C5
:1028C000206011807A69AE331E80012A2BD17A6B89
:1028D000331C396D8B4209DAF86B5900415A108864
:1028E000884200D2118001330232F2E73A6C786BF1
:1028F00053001A5AF96C131C8A4200D20B1C9BB26B
:102900007021FB640123CB557422BB6C0020D05393
:1029100072217122D355CB5573220223391CD35512
:1029200070317A6B10E0786D00F002FF391C80B2D4
:1029300078310222F864B86C0123CA70FA6B4870CF
:1029400088708E800B70301C03F0FCF9386C882383
:10295000D8537A6AFB6B8A214400CA531C19FA6C5B
:1029600023888E21CA538C20391C8031C353042301
:102970004B708B70002502233A1CCB708832B22337
:102980000126281C8D800E700B7103F0DBF9238863
:102990000F4C2268111CE83109680988994224D239
:1029A00006F076FD051C06F0C7FC03787865002B61
:1029B00010D0301C03F008FA23687E6DE83302362D
:1029C0001E6023E0D1250000040E0020FFFFFF7FE2
:1029D00040000020002D19D1164B1B68DB7C002B1A
:1029E00014D1301C03F0E4F910E0E7321278002A29
:1029F0000CD0114E306842889A4207D9281C03F047
:102A0000E3F923683268E83302321A6079690029F1
:102A10000AD17A6AD0B201F024F80848796801F046
:102A200047FDBD4625B0F0BD03F086F8072800D16C
:102A300093E6EEE7000E0020040E0020D1250000F2
:102A4000F0B57B4E8DB0724671460190301C0392FA
:102A500001F016FD06F01CFD041C03F0BBF8071C7A
:102A600003F0C6F8734D02902B681A1CE4321278FA
:102A7000BA4226D0002F0CD000226B469A826946BB
:102A80003B230B75101C04A90492022403F05AF98D
:102A900012E0029A3E1C002A0FD106A93C23381CE2
:102AA0003A1C8F8006970B7103F04CF92B68E633C4
:102AB0001C78631E9C41E4B202262B68E4331F702D
:102AC0001FE01A1CE532127802998A4218D00029B8
:102AD00006D1E6331C78631E9C41E4B23A2301E040
:102AE00039230224002208A9101C8A8008920B7145
:102AF00003F028F92B68029AE5331A70022600E0E9
:102B0000002603F021F8071C03F056F8019B032B65
:102B100002D0002F03D107E00226002F38D000207A
:102B200003F01AF8022633E02B68E4331F88002FE5
:102B30002ED10199012902D0022904D00EE001987A
:102B400003F036F90AE0381C03F032F92B68E7335A
:102B50001B78002B02D0381C03F036F903F022F961
:102B60002B68071CE6331B78834211D0002802D063
:102B70001123012401E01223041C00220AA9101CC5
:102B80008A800A920B7103F0DDF82B68E6331F7020
:102B900006F07EFCA0422AD006F07AFC06F0C0FBCC
:102BA000071C201C06F0BCFB019006F071FC201CE9
:102BB00006F068FC06F030FC1F4B3A1C1B689B3289
:102BC00003CB019B9B3303F0EFFA002001F02AF9BD
:102BD000FEF7BAF9002003F0F7F82B6800211A1C61
:102BE000E7321170154AE833126802321A6006F0B3
:102BF0004FFC06F0A1FB0378002B08D003F0DEF8B1
:102C00002B68E7331A78824201D01870022603F04D
:102C10000BF8041C03F052FF0379A34200D00471A7
:102C20000348039901F044FC301C0DB0F0BDC046D0
:102C3000E12900004000002044000020040E002094
:102C400038B5054C75467146201C01F019FC291C4D
:102C5000201C01F02DFC38BDE12B000038B5054CDF
:102C600075467146201C01F00BFC291C201C01F04C
:102C70001FFC38BDFD2B0000F0B597B000AF7446C7
:102C800071469548BC6001F0FBFB944C6D4623688F
:102C900019685B680A1C5A43D3185B000833DB08C9
:102CA000DB00ED1A8E4B52001B6856084900AA182B
:102CB0004908DD611A62AD46BD6439643E6300F0C7
:102CC0000DFB2168F8638C683D6CBC62827A437AA4
:102CD000BC6C5343DBB27B644B686A005D1E55439A
:102CE000564265197E62BD630020013B0ED3BD6B69
:102CF0000A684519FD64013A05D35400251CFC6C93
:102D000000266653F7E77C6A0019EEE77C6C3D6BA2
:102D1000013CBE6C641964003419BC616C00221C57
:102D2000023ABB69FC61B218934203D000211980BA
:102D3000023BF9E7BD6A7E6CAB005B42FB607B6CDB
:102D40003C6B01335B007D6C5B4276003B617E61D6
:102D50006319BE6C5B00F3181E243B627C63002089
:102D600001F060F85D4A3C6C15685E4B6E68BD63AF
:102D7000311C013949006143FE64BE6C1D68FB6C67
:102D80007118013B29D3BC6B581C2268BC6A9E0099
:102D900054430019520080003A63FE6238600022FA
:102DA000386B824216D0FC6AA8693E6800596C698B
:102DB0007860A0597E680024B04200DD841B8E5AE2
:102DC000A619E410341B8C52FE683C680232A41928
:102DD0003C60E5E77C6A0919D3E7424B00241D6893
:102DE0003E69023CB44219D0E969FA6B78693963EB
:102DF000517A0619786C06F095FB3B6B7600F25819
:102E0000C9B22E6A89008B593E6AD31ADA43D217A7
:102E10001340325B9B10D3183353E1E77C6B013CCA
:102E20007C63002C9BD1FD6CBE6C7D64FD69BC692C
:102E3000023D7519AC421AD020881E2106F02EFBE7
:102E4000023C6080F6E720881E2106F027FB7B6CA1
:102E500086B2F86C013B2680984205D1301C1421C3
:102E600006F06AFB36182680023C013DEBD2FC6C72
:102E7000013CFC640AD3FE6C3B6CBC6B734325685D
:102E8000BE6C6C1EE41864003419EEE7FFF7E6FE32
:102E9000124D50262B68512118681A791B69F0557C
:102EA0005426F35555200223C3555224381CCA55C5
:102EB000E255B96C002453255030EC5502F0E8FC83
:102EC000074B05481B68B968DC611C6201F0F0FA29
:102ED000BD4617B0F0BDC046192C0000D403002039
:102EE000440000204000002038B5054C754671466E
:102EF000201C01F0C5FA291C201C01F0D9FA38BDAC
:102F0000892E0000F0B58DB000AF7446714642487E
:102F1000FC6001F0B5FA00F0E1F9404C6D46236821
:102F200044CB724393195B000833DB08DB00ED1AD6
:102F3000AD46281C7D623A4D69462B685200D86127
:102F400050088A181A623862002000F06BFF760081
:102F50002168344A760876000B6810687242BA61BC
:102F60005A1E56438446786A86197E6100205C1E8C
:102F7000FC6118D37C694A6804193C61013A0ED39C
:102F800055007D608D683C695D4355196E1CB50028
:102F900066467669AD592E1C7D686653EEE7BA69C0
:102FA000FB698018E3E73D6A7E6A1E4A0B696C0084
:102FB00036191068B4469A00043A013B05D3C46937
:102FC0005900A55866467552F6E7FFF78DFF134C7A
:102FD0002825236829201E681A791B69EE552C259F
:102FE000C255EB552A21381C7E23CA5500242B22BA
:102FF0005B42796A2D262830D455F35502F048FCFF
:10300000074D05482B68F968DC611C6201F050FA35
:10301000BD460DB0F0BDC046A52E0000D403002073
:10302000440000204000002038B5054C754671462C
:10303000201C01F025FA291C201C01F039FA38BDAA
:10304000C92F0000F0B591B000AF744671469048AA
:10305000BC6001F015FA00F041F9FDF7CFFE8D4B91
:10306000F8621C686946656820683D6268434219D9
:10307000D31D5200DB080832DB00D208C91AD20087
:103080008D46891A786268468D4638636846C01A4C
:103090008546814B6D461B68F961BD61796A3D6B60
:1030A000E2685D62281C6D189D62002106F006FB37
:1030B0002269281C002106F001FBE2680021684615
:1030C00006F0FCFA786A22696844002106F0F6FAF4
:1030D0003C6A7D6A63005B083B616B005B08FB60D8
:1030E000FB6A31331B787B637D6B6A4C002D00D10A
:1030F000A9E0002000F096FE684A20681168436845
:103100008C46013B50D30268511EFAD38468654651
:1031100062439A186D69013292005259FD69BA6290
:103120003A694A439A185200545FBA6AFF25A41AB2
:10313000FF2C02DCE543ED172540FA6A7D6033324F
:103140001278BD697A61EE183A6A7D694A43AC42E9
:103150000DDDB45C0134E4B2B454FE6A64B23236BC
:103160003678B44217DB3D6BEC187D6812E0FC6AE0
:10317000B65632342478A6420DDA3D6BEC18A65CC4
:103180007D68B54200DA351CA554BC690025E218FB
:103190003C6A4C4315553A69BC6A4A43FD699A1822
:1031A000520054530A1CAFE73C4A0369FD68166895
:1031B0005A1E5219FC695200A218013B3FD3F5690F
:1031C00099004959B962BC6A0021505E001BFF2872
:1031D00002DDFF257D6103E0C443E41704407C6108
:1031E000F96ABC69333109787D6A8C46611960459A
:1031F0000EDDC85C0130C0B2C854F96A40B2323149
:103200000978884217DB3C6B61197D69CD5412E067
:10321000C8568446F86A3230007884450BDA3C6B35
:103220007D6A6019C45CA4467C69644500DA644622
:10323000C4540020C854BD6A023A5580BDE77C6B77
:10324000013C7C6350E7FFF7EFFE23683A251A79CB
:10325000196839241B69EA55E25538207C6B3C25F6
:10326000C155EB553B207F23C4555B423D20C355E0
:10327000381C396B383002F00BFB074B04481B68D5
:10328000B9685C629C6201F013F9BD4611B0F0BDF3
:10329000E52F0000D403002044000020400000205F
:1032A000014B18607047C04640010020014B186870
:1032B0007047C04640010020014B58687047C04627
:1032C00040010020014B98687047C0464001002033
:1032D000014B18607047C046100E0020014B186863
:1032E0007047C046100E0020014B18607047C04662
:1032F0000C0E0020014B18687047C0460C0E0020D1
:10330000014B18607047C046080E0020014B18683A
:103310007047C046080E0020014B18687047C04631
:103320000402002010B50D4B00201B78AA2B12D1EF
:103330000B4B1C780B4B64B218780B4B40B21978CE
:103340000A4B20181A780A4B49B21B78401880188B
:10335000C01A43425841C0B210BDC04650000200DE
:10336000510002005200020053000200540002000B
:10337000550002008023DB020022188059809A80C9
:10338000C046024B188880B27047C0460600040051
:1033900013B5094A042413780021DBB21C430191C0
:1033A0000198F421FF31884205DC1370C046147087
:1033B00001990131F3E713BD0D00005082B00022E6
:1033C000019201AB55221A70392252429A700122A1
:1033D000DA70019AA023DB059A6102B07047A0233E
:1033E000DB059869C001C00F70470122A023DB05EF
:1033F00010400206024998690840104398617047DE
:10340000FFFFFFFE82B00022019201220A408918CC
:1034100001303F2201AB1040C9B21870481C023184
:1034200002408900D9705A70019AA023DB05DA6145
:10343000196A024A0A401A6202B07047FFCFFFFFC2
:103440000002064B000A0138002258609A600522EB
:103450001A60C0461A68D103FCD5704710E000E03E
:10346000F0B5514F85B03B6894339A7819681D7850
:10347000DE780F231407994312092D0701922D0FAF
:103480000B1C80222B4352001343484A0395484D9E
:103490001340484A2B4048491340240F0B400199E0
:1034A000220413430A0545493607360F0B400096A0
:1034B00013433206424E029433401343414AA02440
:1034C000E4051340E360FFF763FF3B68E268953370
:1034D0001B781540DB069B0FDB021D43E560E268AD
:1034E00080239B001343E360E26880239B01134326
:1034F000E360029C039DFFF715FF002813D0324FB5
:10350000882039781E34C9B206F016F83978444359
:10351000C9B2882006F010F80F3545431E3C002341
:103520000F3D9C4203DB231E0F2B00DD0F230F22D8
:10353000954200DD151CA024E4051F491A40E368EC
:1035400012040B401343E360EB43E268DB171D40BA
:103550000F239A431D401543E560E368F02293432F
:1035600080221343E360E368144A18481340E36081
:10357000E3683340E360FFF763FFE26880235B05A5
:103580001343E3600099E2680B0616401E43E660B1
:103590000F48FFF755FF019B08491A05E3680B40E8
:1035A0001343E36005B0F0BD0C0E0020FFF9FFFFF0
:1035B000FFE7FFFFFFDFFFFFFFFFF0FFFFFF0FFF52
:1035C000FFFFFFF0FFFFFFEF54000200FF0F0000BE
:1035D000FF6F0000064A074B12680120E8321268AC
:1035E00019789040021C0A43D2B21A707047C04644
:1035F00004020020290000500549064B09681A788A
:10360000E83109680120884082431A707047C0463B
:103610000402002029000050044B1878044B1B685A
:10362000E8331B68184101231840704729000050F7
:1036300004020020A0230122DB055A707047044BCE
:1036400082B0019001AA188092789A7002B07047F7
:103650002400005007B500F043FF064B019001AA7B
:10366000188092789A70044B00221A70034B012242
:10367000DA7707BD24000050000000200800005049
:10368000034B00221A70034B0122DA777047C046C1
:10369000000000200800005072B6084B1B5C002B95
:1036A00003D1C04662B630BFF6E762B6A023DB05A1
:1036B0009968034A0A409A607047C046000000209B
:1036C000FFFFF9FF72B6074B1B5C002B02D1C0460F
:1036D00062B6F7E762B6A023DB059968024A0A40A2
:1036E0009A60704700000020FFFFF9FFA023DB0570
:1036F0005A680121120E58689143034A0906024094
:103700000A435A607047C046FFFFFFFE08B5074BEB
:103710001B681A1C9C3212789D331B7852000132B0
:103720005043994005F008FF08BDC0460C0E00202C
:1037300008B5044B1B689F33197849000131FFF726
:10374000E5FF08BD0C0E002008B5A0230120DB0515
:103750005870FFF7A1FFFFF7C9FF08BDF7B5A02616
:10376000041CF605042807D1554B1B681A1CA4320B
:10377000A83317681B6824E0524B1B681A1C8C3353
:103780001B68883217687361FDF74AFBE7300378DE
:10379000002B17D005F07CFE05F0CEFD01797F22CD
:1037A00011408904019171690B1C47490B40019933
:1037B000194371614179444B0A40716992040B408D
:1037C00013437361A023DB051F611E691F231E4085
:1037D000FFF7A8FD00280AD03C4B88201978043652
:1037E000C9B205F0A9FE46430023043E03D4331EAC
:1037F0001F2B00DD1F23A022D205108A1F210B40A2
:10380000884303431382022C16D007DC002C13D00C
:10381000012C2DD12B4B1D689E3529E0042C07D09F
:1038200023DB052C24D1264B00241D68AF351FE077
:10383000234B1D68AC351BE0FDF7F2FA031CCC33BB
:103840001B78002B03D01E4B1D685D3510E0E73060
:103850000378002B05D005F01BFE05F06DFD851DDE
:1038600006E0184B1D689B3502E0164B1D68A1351C
:10387000A023DB05596928783F221040914301437A
:10388000596168781F215D6908401149C0022940CB
:10389000014359610F49640009680C19211C7731F3
:1038A0000878596810409143014359607834217871
:1038B00058680A401102084A02400A435A60F7BD9C
:1038C000100E00200C0E0020FFFF03FE540002002B
:1038D000FF07FFFF04020020FFC0FFFF294BF0B5E8
:1038E0001A68294B85B01B689E331B785B069B0EBC
:1038F0000193931DD97F00238D005519581E5B1825
:10390000002B27D053181B1826331B788024D3187C
:103910005E78A023DB055F68E4033C435C60019CA8
:10392000B606240400945F68B60EBC46174F644682
:103930002740009C27435F60C04624367600840001
:10394000F65A2C19983426605E68114C34405C603D
:10395000031CD3E76F460293BB8101233B72931D87
:10396000DB7F7F217B72BB72FB7A98328B43042111
:103970000B43FB720F20B02302A93B7302F0E2F964
:1039800005B0F0BD040200200C0E0020FFFFC0FFB8
:10399000FFFFBFFFF0B585B0FFF7A0FF154B002577
:1039A0001E68B31DDC7F631C9B005B420093A30079
:1039B000F3180193009B043D9D4208D0019A012118
:1039C000571998373868FFF7A1FE3860F2E76A4662
:1039D00000239381012313720423D372B023547202
:1039E00094721373321C98320F2002A902F0AAF9C4
:1039F00005B0F0BD04020020044B00225A70A02341
:103A0000DB055A7001221A707047C0460000002082
:103A1000A023DB059968064A0A40802189020A43EF
:103A20009A60044A0021917001229A707047C04642
:103A3000FFFFF9FF00000020024B1B68903318685D
:103A40007047C04604020020024B1B689033186088
:103A50007047C04604020020A023DB059868C0B26E
:103A6000704730B5A023DB059B68DBB283420ED0E4
:103A700001DA013300E0013BA022D2059568FF2165
:103A80001C1C8D430C40291C21439160EEE730BD86
:103A9000A023DB059968802252020A439A60996844
:103AA000094A0A409A609A68120112099A60D96814
:103AB000064A0A40DA60D968054A0A40DA60D968DD
:103AC000044A0A40DA607047FFFFFFF0FFFEFFFF85
:103AD000FFDFFFFFFFFFFFEF1B4B10B51A6801214F
:103AE000131C92331878A023DB059C680840174903
:103AF0000004214001439960933210789C68144976
:103B00000007000921400143996011789A6809096A
:103B10001201090712090A439A60D96880225200EB
:103B20000A43DA60D968802292010A43DA60D968D0
:103B3000802252050A43FA20DA60800000F0F4FC8B
:103B4000FFF77EFC10BDC0460C0E0020FFFFFEFFFD
:103B5000FFFFFFF008B50020FFF79EFD08BD034BF7
:103B60001B689C3318784000013070470C0E002011
:103B7000024B1B689D3318787047C0460C0E00201E
:103B80000048704700100050004870470020005067
:103B90000048704700400050074B01201B685B79CC
:103BA0009A1C0340D318054A1268663210785843AD
:103BB000034B8000C0187047100E00200402002044
:103BC00004400050F7B51B4B051C1C68A3795F1E11
:103BD00015D36279013A10D36079561C811C01918A
:103BE00001210840019908185843311812488900EA
:103BF00009180868E8400860ECE73B1CE7E7FFF7B6
:103C0000CBFFA37A002201339C466346013B9C46CE
:103C10000FD3617A96000191861900230199994288
:103C200005D09F00F1590133E940F151F6E75218F0
:103C3000EBE7F7BD100E002000400050074B0120BD
:103C40001B685B799A1C0340D318054A12687232CC
:103C500010785843034B8000C0187047100E0020A6
:103C60000402002004400050094B01211A685379D6
:103C7000D0799A1C0B40D318064A013012686A3278
:103C800012785343C018044B8000C0187047C046D8
:103C9000100E00200402002000400050F7B5434BF6
:103CA0001D682A7853B2042B1DD1414B19680B1C97
:103CB000AE331F7802235E1E77D34A79013A10D3C0
:103CC0004C79551CA01C0190012004400198041956
:103CD0005C432819374C800000190468FC400460DC
:103CE000ECE7331CE7E7002A45D0022B21D1FDF792
:103CF00097F8CC3003782E4C002B02D023685F332A
:103D000002E02D4B1B689D331878FFF75BFF256899
:103D1000EC79002C2FD0FFF7A7FF061C013C2AD31B
:103D2000697A201C05F05EFC89008A59A300F250D4
:103D3000F4E7032B03D1204B1B68A33318E0012BBE
:103D400011D1FFF77BFF1A4B061C1B685C79013C05
:103D500011D32B193A331B789B009859FFF7E8FCD5
:103D6000A300F050F3E7052B05D1114B1B68B133CD
:103D70001878FFF727FF104B1B689A331B78002B2E
:103D800013D00B4B1A685379013B0ED3517901259F
:103D90008C1C294061189479581C614340180549CE
:103DA0008000401800210160EEE7F7BD040200200A
:103DB000100E0020004000500C0E002008B5A0237B
:103DC0000120DB055870FFF767FCFFF78FFCFFF75A
:103DD00065FF08BD70B5041C104E114D11D10120B6
:103DE000FFF7BCFC336801221A70A023DB056C705E
:103DF0005C701A70FFF7E2FFFFF778FCFFF7CAFD6F
:103E00000224201CFFF7AAFC336800221C70A023A8
:103E1000DB056A705A7001221A7070BD040200201E
:103E20000000002008B5FFF7D5FFFFF7C7FF08BD6A
:103E300008B5A023DB05011C58683F2211409043C0
:103E40000843586059685868114001310A4011020E
:103E5000064A02400A4306495A6000224A705A70D4
:103E600001221A70FFF7AAFF08BDC046FFC0FFFF7E
:103E70000000002010B5A023DB051C6A0005064ADF
:103E8000000D010422400A431A621A6A120B12033F
:103E90001043186210BDC046FFFF00F073B5174B0A
:103EA000A0221B68D20590339168196891601C7834
:103EB000FFF738FA124D002812D0124B124A1B7825
:103EC00012782E6852B25BB20092201C1021D122CF
:103ED00001F0F2FF2B689436306094331B68E418CD
:103EE000002C01DA002402E0FF2C00DDFF242B6807
:103EF000E0B290331C60FFF7B4FD73BD0C0E0020E0
:103F000004020020530002005200020008B5FFF72F
:103F1000C5FFFFF7A5FAFFF751FA234BC022920025
:103F200098582249014099509958FF2081434020D8
:103F30000143995098581E490140802000040143D4
:103F40009950985880210002000A090601439950AF
:103F5000012102221A6008201960042119601860EA
:103F6000144B00205860144B186901431961134B1E
:103F70001B68197A124B1B68E833002900D1032211
:103F800010491A6000230B700F49A0220B700F49D3
:103F9000D2050B709363D36B9B0E9B06D36362B603
:103FA00000F09CFE08BDC04600E100E0FF00FFFFFE
:103FB000FFFF00FFFCE100E000ED00E0100E00203C
:103FC0000402002029000050280000502A00005060
:103FD00008B5002801D0012801D100F07FFEFFF7CD
:103FE0005DFFFFF73DFAFFF7E9F908BDF0B5214B9A
:103FF00013211B680224DA7A0023133AD2B29142C9
:104000005B41E41AA023DB0558693F225968104040
:104010008022D2030A43A3B05A60411EA023C9B232
:10402000DB0502AAFF2910D05F683F26124D0E4023
:1040300036043D4035435D60C046251C24356D0087
:104040005D5B4B00D5520139E8E75C680B492140C4
:104050005960694600238B8001230B70022348704E
:104060008870CB700320B3230B7101F06BFE23B07B
:10407000F0BDC046100E0020FFFFC0FFFFFFBFFFD6
:10408000F7B5041C02F008FD124B1A6800235068B3
:10409000411C0191019D16689D420CDB9768013619
:1040A0007E4399008C469E1900216546B6006151F9
:1040B00001333151EEE701239E420ADB956800216E
:1040C0005D43AF002D180135AD0039510133295141
:1040D000F2E7F7BDD4030020044B054900221A6023
:1040E00059609A6005221A607047C04610E000E0EF
:1040F000FFFFFF0010B5A023DB059C6899680C4BFF
:10410000C9B21B68E40394331B68E40F591AFF31EA
:10411000E62359430134074BA040C918041C064844
:1041200005F00AFAC1B2201C05F006FA10BDC0461F
:10413000040200205C5D000040420F00014B0022A1
:104140001A60704710E000E030B50E4D0E48AB68C5
:1041500085B0C01A0193FFF7CDFF02A90123002407
:104160000B704B708B7004230190CB70201C6F235D
:1041700001AA8C800B7101F0E5FD01982C6005B05F
:1041800030BDC04610E000E0FFFFFF0010B5041C8A
:10419000FFF7A2FF201CFFF71DFEA023DB05012077
:1041A0005870FFF78FFAFFF7A1FAFFF777FDFFF7D7
:1041B000CBFF10BD37B5051C0424291C221C684602
:1041C00005F03AFA2919221C01A805F035FA0099E0
:1041D00080230ABADB05DA6001990ABA1A6137BD91
:1041E00040BA80B2704700BA70470023114A1249A2
:1041F0009A188A4204D21149C95804331160F5E76C
:104200000F4B104A191D043B934203D200221A603F
:104210000B1CF6E70C4B0D4A1360EFF308820433D6
:10422000191D043B9A4203D9094818600B1CF7E793
:104230007047C04640000020E8030020349800008A
:10424000EC030020000E00204C0E0020280E002061
:10425000CDCDCDCDF0B5294D89B029482C6800F0E1
:1042600063F9FFF7EDF80026264FBC4222D28037D3
:104270003B1B2027832B00DC9F1002A9FAB20123ED
:1042800000204A708A70BF10221C0B70CB7088808F
:1042900001F058FD231C3A1C013A08D3002E04D12A
:1042A00019491868884200D01E1C0433F4E7BF0087
:1042B000E419D9E72B6804A9F31A00250193042314
:1042C0000124CB70281CA72301AA8D800C704C7090
:1042D0008C700B71843701F035FD06A90420C8707D
:1042E000A823BE1B281C01AA8D8001960C704C705F
:1042F0008C700B7101F026FD09B0F0BD280E002076
:10430000801A060080370020CDCDCDCD024B1B6832
:104310000633D87F7047C0460402002070B5051CE4
:10432000FFF78CFC0A4B1C68A31DDB7F9A00AD18BD
:104330000022511ED218002A09D0E2185218263243
:104340001278920016588A00AE500A1CF1E770BD30
:104350000402002030B50B4B1B689A1DD27F9400DD
:104360001C195300C01800230133D11A013107D0A2
:104370009D00651B983559002D6849424552F3E769
:1043800030BDC04604020020A02382B080B2DB050D
:10439000D88502B07047A023DB05D88D82B002B06B
:1043A00070470722A023DB0510404201188AE02154
:1043B0008843104318827047F8B50C1C051CFEF7A3
:1043C000A5FF144908688379013B11D30E687279FF
:1043D000013AF9D30E6870790F4E58433668801849
:1043E000F6182818A03607783679BE190670EFE758
:1043F0000B68DB79013B08D3074AE15C1268D218ED
:10440000C83212788A18E254F4E7281C211C00F004
:10441000E1FEF8BD100E00200C0E0020134BF7B586
:104420001C686946E26800AF131C0E33DB08DB0032
:10443000C91A23698D460E33DB08DB00C91A0C4B01
:104440006D461E688D467960281C311C05F0F4F815
:10445000F0239B00F1182269786805F0EDF8281C1C
:104460007968FFF7A9FFBD46F7BDC046D403002019
:10447000080E0020A023DB0518690006400F7047D6
:1044800070B5051CFEF71EFF0468061C013C08D32E
:104490007268E300D3181A68AA42F7D15B6898479C
:1044A000F4E7024B013D1D6070BDC046140E0020B4
:1044B00070B5051CFEF706FF8468061C013C08D396
:1044C000F268E300D3181A68AA42F7D15B689847EC
:1044D000F4E7024B013D1D6070BDC046140E002084
:1044E00038B5A023DB0599689D680C4B041C1B683C
:1044F0000B4894331B68ED03C91AC943E623C9B2BC
:104500005943084BED0FC91805F016F8044B013557
:104510005843211C284105F00FF838BD0402002043
:1045200040420F005C5D000038B5A023DB059968B0
:104530009C680A4B051C1B68094894331B68E403FC
:10454000C91AC943E623C9B25943064BE40FC91837
:1045500004F0F2FF68430134204138BD040200201A
:1045600040420F005C5D0000002801D0133907E0D5
:10457000122902DD262902DD1239491000E000E08F
:10458000081C7047F0B5AA4B00261D68041CEB7A86
:104590001322133BDBB2301C9A427041B1B0C7B258
:1045A000059702273F1A311C142209A805F086F846
:1045B000A04B20681B68882201936B331870019B05
:1045C00061686E3319700EA8311C05F077F8311C44
:1045D000142209A805F072F8974B0EA81968442216
:1045E00005F02AF8022F04D11FA80EA9442205F0D5
:1045F00023F800272E1C0497771B03976B7901364D
:104600009F423EDAB77A0598391CFFF7ADFF09A93A
:10461000095C0EAB0291029A4421514309185918C2
:10462000721B0A717911069109A90A5C11214A438A
:10463000069952181F210F40063201219200B940FD
:104640000F1CD1580F43D7500399019F3F237A186D
:104650005178071C99438C4602991F4089010691A5
:10466000614603970F431F40069B1F43029B5770F1
:10467000013309AFDBB23B54049F9F42BCDA049381
:10468000BAE7019B049D6D3300261D700296684BAE
:10469000029E19688F79BE4200DBBEE0029D491977
:1046A0000B1C2833DA79644B1E68331C9A331B7851
:1046B000B446039303980023984204D0781E8542A1
:1046C00001DA2931CB790120011C91400591111C9F
:1046D0002039051C8D40A9011D1C203D061CA84049
:1046E000049D9E408909069607900195019D002D25
:1046F00038D0019E4425013E7543019666680EA898
:104700002E544519281C002620302E624668B60E0D
:10471000B606009646601F2A02DC0598286204E06F
:104720008D01009EAD092E434660039D002DDDD016
:10473000029E781E8642D9DA019E442575430EA852
:1047400045191F2B04DC2E6A069830432862CDE7FA
:10475000686A079E0643B601800EB609800630439C
:104760006862C3E7029E6046331C45786344C833E1
:10477000AD065F79AD0EFEF7D5FD002813D02F4EA4
:10478000882031780137C9B204F0D6FE317847432A
:10479000C9B2882004F0D0FE02354543013F023DF6
:1047A000019E791C03D03E1E1F2E00DD1F263F2DCB
:1047B00001DD3F2526E0EB43DB171D4022E0019998
:1047C000442251430EAB59188F781F239F43301C4E
:1047D00018403B1C03434F788B703F23281C9F439A
:1047E00018403B1C034320684B703B281CDC5043A3
:1047F000134FC01904F020FF2368019F01330137D4
:1048000023600197019F04988742D8DB029D63686B
:10481000013501330295636039E7064B22681B6856
:1048200001206C331A7000E0002031B0F0BDC046AA
:10483000100E0020040200200C0E00205400020084
:104840000080005030B585B0FEF760FD064B01A832
:104850001B68021C843332CB32C2FFF793FEFFF792
:10486000DDFD05B030BDC04604020020F0B5564B5A
:104870009FB01B6800270493DB7A1322133BDBB243
:10488000391C9A427941CBB2051C391C142208A864
:10489000079304F013FF4D4B2A681E680DAC331CC0
:1048A0006F331A706968023359701F70391C4422C3
:1048B000201C04F003FF391C142208A804F0FEFE9B
:1048C000434B201C1B684422191C069304F0B4FEC1
:1048D000B31DDF77049A53799F4233DA049A07981D
:1048E000D319DB7A191C0593FFF73EFE08AB1B5C5E
:1048F0009C46002B0BD1B31DDA7F511CB218D9771F
:104900000732FBB20DA9D37701330A1813710DAB2F
:1049100019180979F2193A320139117005990137DC
:104920004A110632920003921F220A40012191404F
:10493000039AD2581143039AD1506346013308A910
:104940000B54C7E7069B5E78B606B60EFEF7EAFC88
:1049500000280AD01F4B882019780236C9B204F00B
:10496000EBFD46430023023E03D4331E3F2B00DD04
:104970003F23A2781F218A436178A2703F2291438E
:104980001340626A0B4369686370930E21709B0643
:10499000002119A814222162636204F08FFE2868A6
:1049A000442250430C4B211CC01804F045FE6A6899
:1049B0002B6801326A60054A0133126801207032A7
:1049C0002B6013701FB0F0BD100E002004020020F9
:1049D0000C0E00205400020000800050F0B5BA4BCD
:1049E000B1B01B680024039353331B78071C133B9F
:1049F000DBB21322201C9A426041C5B20595022504
:104A00002D1A211C142209A804F058FEAF4B3E6851
:104A10001B68211C049363331E70049B7868663303
:104A2000187088220EA804F049FE211C142209A83F
:104A300004F044FEA64B0EA819684422443104F049
:104A4000FBFD022D04D11FA80EA9442204F0F4FDA1
:104A50000025039C0695039E039DA61B07966B7A73
:104A600001349E4237DA231C52331D780598291CE5
:104A7000FFF77AFD09AA115C6E118C46029611218E
:104A800066467143029E0EAB89191F2635400631DA
:104A900001268900AE40351CCE583543CD50079EC7
:104AA000049D3F23A919051C1D40583166460295F7
:104AB000B6018D790196029E9D432E431E40019BB7
:104AC000069D1E4363460133DBB28E7113549D4233
:104AD000C1DA0693BFE7069E049BF6B265330796DC
:104AE0001E700024784B04941B68049D9A7A9542AA
:104AF00000DB9BE0049D069C5A1958321178012274
:104B0000081C2038161C82408E409001B446800953
:104B10000394039C002C1BD0039D4422013D6A4357
:104B20007E680EAC1655A2180395141C1F2905DCCF
:104B3000566A65461562B20E920607E000251562B8
:104B4000666A8201B50E9209AD062A436262E0E709
:104B50005E4A1168221C587A824210DA881858304E
:104B600084794425A006A4096C43BE68800E2018F1
:104B70000EAD0136281806710132BE60EBE7544BCA
:104B80001B681A1C4632453316781C78F606A406B4
:104B9000F60EA40EFEF7C6FB002813D04D4D88205C
:104BA00029780136C9B204F0C7FC29784643C9B256
:104BB000882004F0C1FC02344443013E023C00253D
:104BC000701C03D0351E1F2D00DD1F253F2C01DD7D
:104BD0003F2402E0E343DB171C40039E0698864215
:104BE00021DA0399442251430EAB59188E781F23C2
:104BF0009E43281C1840331C03434E788B703F2380
:104C00009E43201C1840331C03433868324E5043E7
:104C10004B70801904F010FD3B68039E0133013690
:104C20003B600396D9E7049C01345BE7274A3E6862
:104C30001468079D221C643216703868D070796839
:104C40000532517015700022597A8A4210DAA11883
:104C50005831897944208D0689094843AD0EB968D9
:104C600040190EAE0131301801710132B960EBE725
:104C70001AAD03950025069EB5421EDA44236B4308
:104C80000EA8C618706A0021820E92063162726206
:104C90000398142204F012FD3868442148430E4A58
:104CA000311C8018442204F0C7FC3B68039E01338A
:104CB00044363B6001350396DDE73B6868340120EC
:104CC000237031B0F0BDC046100E00200402002059
:104CD0000C0E00205400020000800050F0B56B4B19
:104CE00000241F681322FB7A211C133BDBB28DB01A
:104CF0009A4261410226CBB20C22761A04A8211CEA
:104D0000019304F0DBFC142207A8211C04F0D6FC5C
:104D10007A793D1C02920299EB1B8B4213DAE97AF5
:104D20000198FFF721FC132801D90020ACE007AA65
:104D3000135C0135B342F8DA0133DBB213549C4201
:104D4000E9DA1C1CE7E701220492B87900218142CC
:104D50000ADA131C9D1AA54203DA3B2BE5DC01336A
:104D6000F8E701311A1CF2E70492FB79002B11D10C
:104D7000002304A80493FFF779FD04A8FFF702FCC1
:104D8000424B434D1B68DE79002E3ED004A8FFF74E
:104D900025FE50E03B1C53331B780025133BDBB250
:104DA0001322291C9A426941CAB202920222521A63
:104DB000019207A8291C142204F080FC7B7A3E1C77
:104DC0000393039AF31B934214DA331C5333197879
:104DD0000298FFF7C9FB1328A7D807AA135C01990B
:104DE00001368B42A1DA0133DBB213549D42E8DA7B
:104DF0001D1CE6E7EB43DB171D40BB7A5D43049BBC
:104E00006D00ED183B2DB3DD8FE72868311C0422BF
:104E1000633004F053FC2868311C0422673004F02E
:104E20004DFC2B680499CAB2191C633168330A70AF
:104E30004A700A711A702D6864002B1C6F331A783F
:104E4000073BDA73291C1B7878310B704A700839DC
:104E500009782A1C7A3211700F3A1678291C7B3196
:104E6000281C0E707D305374022204F0E5FB2F1CC9
:104E70002B1C7F33083734195C701E706E35FE674B
:104E80002A7801339A6001200DB0F0BD100E002089
:104E9000040200200D4B10B51C680D4B01681B6807
:104EA0001A1C673211704168D170191C69310022D7
:104EB0000A70617A8A4204DA8168013201318160C4
:104EC000F7E70268683301201A7010BD100E002049
:104ED00004020020A14BF0B51B68B3B01A1C0832C5
:104EE000D26F002406929E4A13211568201CEA7A8C
:104EF000069F133AD2B2914260411A1CC6B2733275
:104F0000177076330296012202261A70361A211C77
:104F1000882210A804F0D2FB211C14220BA804F054
:104F2000CDFB291C603110A8442204F085FB022E21
:104F300004D121A810A9442204F07EFB6E79002739
:104F4000059603973C1C059FBC422ADA2B19DE7A92
:104F50000298311CFFF708FB0BAB195C10AA8C46BA
:104F60006746442179430918511801340C711F5CBC
:104F70007111049111214F4304997F18B91D1F2706
:104F80003E4001278900B7403E1C8F583E438E505B
:104F900062460132039ED2B21A549642D3DA039289
:104FA000D1E7069D00240595039F0297029F002FDD
:104FB00016D0029E4422013E724310AFBA180296E8
:104FC000D66A0021556A11629162B10E8906D378C2
:104FD000A80ED162202180060B435062D370E5E712
:104FE0005F4B221C1868817984460791079D131B2B
:104FF000AB4248DA65462B1B9B182F3318780123E8
:105000001F1C874051100497071C1940203FE6B22F
:105010000991BB40039908961F1C002931D0013922
:1050200044234B4310AE651C9D55089DF318099E03
:105030006DB20195B54210D01F2804DC1E6A049D94
:1050400035431D62E9E75D6A2E1C3E43B601AD0E95
:10505000B609AD0635435D62DFE71F2804DC9E6AB2
:10506000049D35439D62D8E71D1CDB6A3B439B01D1
:105070009B090193EB6A9E0E019BB6063343EB62DC
:10508000CBE70132B2E7374B1B685B19C8335F7956
:10509000634661331D78AD06AD0EFEF743F9002877
:1050A00013D0314E882031780137C9B204F044FA68
:1050B00031784743C9B2882004F03EFA02354543AF
:1050C000013F023D0026781C03D03E1E1F2E00DD4E
:1050D0001F263F2D01DD3F2502E0EB43DB171D407E
:1050E000059944274F43214ABF18029A039B9A42CD
:1050F00020DA02994422514310AB5918301C1F2367
:105100001840049088789843031C049803438B70DC
:10511000281C3F231840049048789843031C0498A7
:1051200003434B70381C04F087FA0299443701316D
:105130000291DAE7DB43039D059EDB172B40F6184F
:1051400001340596022C00D02EE7044A069D126811
:10515000E918CB187432137033B0F0BD040200208C
:10516000100E00200C0E00205400020000800050A1
:10517000F8B5164D061C2B68002463331F782B6886
:10518000E1191A1C643212780134914209DAE319E8
:10519000442058430E4B311CC018142204F08EFAE0
:1051A000EDE76B331F7800242B68E2196C331B7812
:1051B00001349A4209DAE31944205843044B311C64
:1051C000C018142204F07AFAEEE7F8BD04020020B9
:1051D000EC7F0050F0B5374B85B01B6802901A1C6D
:1051E000039163321578344A00201168041C8A7ACE
:1051F00094422BDA021C4F7A161ABE421FDA9E190D
:105200005836B679B7090096EF1944267E432B4FDE
:10521000B4463E1C009F66440196BE06039FB60E30
:10522000B446BE5C3F2E00DD3F26F6B20096019EDE
:105230000132371C6744009E30373E70DBE7181C94
:105240006530007801342D18101CD0E71A1C6B3221
:10525000147800208A79904229DA00224D7901954C
:10526000AA421EDA9E187678B709E71903974427F1
:105270003D1C039FB6067D43AC46104DB60E2F1C59
:10528000019D674445430397029FBF187D5D3F2DF5
:1052900000DD3F25039FEDB2BE1930363570013277
:1052A000DCE71A1C6D3212780130A418D2E705B081
:1052B000F0BDC04604020020100E00200080005007
:1052C00044235843044B111CC018C2780F231940C3
:1052D0009A430A43C27070470080005038B5051CDD
:1052E000141CFEF71FF8002808D00A4B88201978F4
:1052F0000234C9B204F020F94443023C442068431C
:10530000054A3F23801802781C409A4314430470D6
:1053100038BDC046540002000180005010B5041C86
:10532000FEF700F8002808D0084B882019780434CC
:10533000C9B204F001F94443043CA023DB05198AF7
:105340001F22144091430C431C8210BD54000200E4
:1053500030B50F4B1B689979884203DA1B18283344
:10536000D87914E05A798D18411AA84202DA5B18EC
:10537000D87A0CE09C7A8A1A2D19A84203DA9B1875
:105380005833187803E0141B1B195033D87830BDFC
:10539000100E0020F0B5D44DA024E405A3682B68BE
:1053A00097B059799A7900AF8A18597A9B7A52182E
:1053B000D3181A1C5A437B62D31DDB08DB006846F6
:1053C000C01A85466B46FF217B6104F077F9FF2008
:1053D000FFF7AAF8C54B69461B1A786ABB60C00084
:1053E000031C0E33DB08DB003861C91A786A8D466E
:1053F0006B4680003B62031C0A33DB08DB00C91AE2
:10540000002200233A637B63F860F961E268B84BDD
:105410008D461340E3602B685C79B34B013C1B68FD
:10542000621C14D01B19381CD97A5030202204F089
:10543000E5F83D6D58207A6DAB00C019C318012105
:10544000283B91400A1C19680A431A60E5E79C79D9
:10545000A54B013C1B68621C15D01B192833381C56
:10546000D9795030202204F0C9F83D6D58207A6D6A
:10547000AB00C019C3180121283B91400A1C1968D0
:105480000A431A60E4E75C7A974B013C1B68621C94
:1054900015D01B195033381CD9785030202204F015
:1054A000ADF83D6D58207A6DAB00C019C3180121CD
:1054B000283B91400A1C19680A431A60E4E79C7A69
:1054C000013C621C17D0884B381C1B6850301B19DC
:1054D00058331978202204F091F83D6D58207A6DE8
:1054E000AB00C019C3180121283B91400A1C196860
:1054F0000A431A60E4E77D69BD610025FD62FD6A2B
:10550000786A854200DBDEE000213A69386A04F0FF
:10551000D5F8A0240021FA68F86904F0CFF8E40572
:1055200000232363636B9B0E9B0663633D6BA56344
:10553000786BB862E36B86019B0EB6099B0633431A
:10554000E3636420FEF7F0FFFDF77AFFF86AFFF7E8
:10555000FFFEC1B2381C4830202204F04FF8396BEE
:105560007A6BFB6CB963FA63BA6C012199405820DD
:105570000B1CC01991004118081C203802689A437E
:105580000260B86C131C00280AD028390A685340FE
:105590009A01636B92099B0E9B061343636301E0C0
:1055A0006B402363A024E405A563E36B0A209B0EF4
:1055B0009B061E43E663FEF7B7FFFDF741FFE26B74
:1055C0008023DB041343E363B96BBA6A4D40A563E0
:1055D000FB6B5A40E36B92019B0E92099B061343AF
:1055E000E363FEF779FDFD6BBE6B3B6AAC460124BD
:1055F000404ABD689168A94214DB3F4A654610687D
:10560000526830402A405D68954203D3F0D11D684E
:105610008542EDD2FD69DA60A2009860A95001349C
:105620000833E5E7FEF78AFDA023DB05D96B334A93
:105630000A40DA63012C3ED0651E386AED00451938
:10564000013C002C37D02B1C083B1A6829685B688A
:1056500091436A687E6A9A43A30039647A64013E82
:10566000BB62FA6A964224D0301CFFF771FE011C1F
:10567000381C5030202203F0C1FF7B6D0122386DB1
:105680009A405821131CC91982008A18183A1268C6
:105690001A420CD0BB6AFA691720D25840425043D4
:1056A000174BC018FEF726FDB96900118855013E59
:1056B000D7E7083DC4E7FD6A786A0135FD62BD6938
:1056C0002D18BD611BE7C3B2381C50300370437006
:1056D00083700023C370037179690123437100F063
:1056E000D7F8BD4617B0F0BD100E0020FFFFFF0039
:1056F000FFFF0FFF10E000E040000050FFFFFFFB46
:10570000E9FFFF16014B18607047C0461C0E0020D1
:10571000014B18687047C0461C0E0020014B1860F2
:105720007047C046180E0020014B18687047C046ED
:10573000180E0020014B18687047C0460802002070
:10574000F7B52F4F73467146381C0193FEF798FE4C
:10575000FBF754FB009001F09FF9061CFDF7BEFD1E
:10576000284D1022041C0099286803F065FF328838
:105770002B68381C1A74120A5A74B2889A74120A66
:10578000DA74214A12680532D27F002A03D0A27946
:105790001A75627902E062791A75A2795A75E2790E
:1057A0009A751A4A6B6812881A70120A5A70184A47
:1057B00052889A70120ADA70164A52881A71120ABE
:1057C0005A71154AD2889A71120ADA71134AAB6873
:1057D000920A1A70124A920AD2B25A709A70114AF8
:1057E000920AD2B2DA701A710F4A920AD2B25A7180
:1057F0009A710E4A920ADA710199FEF759FEF7BDC5
:10580000E15600000C020020D4030020FE0300003B
:10581000FC9B0000FCAF0000F8BF0000000000008F
:1058200000040000009C000000B0000000C0000068
:10583000F7B50A4C7146061C201C7546FEF720FE83
:10584000074A694681CA81C16B46B600F658201CDA
:10585000291CFEF72DFE301CFEBDC046D1570000AE
:105860000897000070B5084C7146201C7646FEF77C
:1058700007FE064B201CDB69311C5D78EDB2FEF79C
:1058800017FE281C70BDC046055800000C02002001
:10589000F8B5144D041C0F1C281C71467646FEF703
:1058A000EFFD114BFF215A6A117010499C620F6085
:1058B000A0782778596B474320793F1860794006D4
:1058C000400E784308609869A0210170D969281CAE
:1058D0001378FF2B02D10B78022BF9D0311CFEF785
:1058E000E7FDF8BD315800000C0200201C05002027
:1058F00038B50D4C7146201C7546FEF7C1FD0B4AAC
:10590000D1694B780A49DBB20B72012B05D0022B0F
:1059100005D1936901225A7001E0FDF75BFE291C55
:10592000201CFEF7C5FD38BD915800000C02002078
:105930001C05002038B50D4C7146201C7546FEF73D
:105940009FFD0B4BDB68002B0BD00A4ADBB2106CBF
:105950007F21194048320170937001335370FFF773
:10596000C7FF291C201CFEF7A3FD38BDD558000039
:105970001C0500200C02002070B50F4C7146201C45
:105980007546FEF77DFD0D4B261C1B7A0C4C012B3A
:1059900005D0022B05D1A2690023537001E0FDF769
:1059A0002BFE236C7F211A78301C8A431A70291C25
:1059B000FEF77EFD70BDC046195900001C05002091
:1059C0000C020020F7B51E4E7346301C7146019341
:1059D000FEF756FD1B4D00241B4E337A012B07D0DA
:1059E000002B18D0022B17D1184B9B695C7813E061
:1059F000FDF712FE041C002D0BD1FDF7FDFD2E233B
:105A0000FF33013B002B01D0C046FAE7FDF7E2FD72
:105A10000C4D013D00E01C1C0C4FFA695378327AA2
:105A20009A4206D0FFF7A8FFFB69074A5B7813721A
:105A300001E0002CD0D102480199FEF739FDF7BDF5
:105A400065590000FF2C01001C0500200C020020FD
:105A5000F7B5164D7346071C0E1C281C71460193A2
:105A6000FEF70EFDFFF7AEFF114C8022236C524271
:105A70001978606C0A431A70391C321C03F0DCFD83
:105A8000236CF6B218787F229043311C1140021C1F
:105A90000A431A704834A670FFF72AFFFFF792FFF7
:105AA000281C0199FEF704FDF7BDC046F15900001E
:105AB0000C020020F8B5FBF7A1F900F0EDFFFDF7AF
:105AC0000DFC1A4C051C666B03F018FC7060FFF7A8
:105AD00037FE174B1B681888E36B020A5A7118715E
:105AE000FFF7A6FEE26BC6B296712B68EF7901361E
:105AF000FF1801374743381C00F0EFF93A1C00212A
:105B0000051C206403F0DAFD231C48330135002214
:105B10005E7065649A7003F0EBFB064B5860A0233F
:105B2000DB059A7CE36C1A70F8BDC0460C020020BD
:105B30001C0E00201C050020024BDB691878C0B247
:105B40007047C0460C020020024BDB699878C0B257
:105B50007047C0460C020020014BDB69987070470B
:105B60000C020020024BDB69D878C0B27047C046F7
:105B70000C020020014BDB69D87070470C0200203A
:105B8000014BDB69586870470C020020024BDB694F
:105B90005A6858607047C0460C020020024BDB690F
:105BA000187AC0B27047C0460C020020014BDB6976
:105BB000187270470C020020024BDB69587AC0B2A1
:105BC0007047C0460C020020014BDB6958727047D9
:105BD0000C020020024BDB69D87AC0B27047C04685
:105BE0000C020020014BDB69D87270470C020020C8
:105BF000024BDB69987AC0B27047C0460C020020A5
:105C0000014BDB69987270470C020020024BDB6984
:105C1000187BC0B27047C0460C020020014BDB6904
:105C2000187370470C020020024BDB69587BC0B22E
:105C30007047C0460C020020014BDB695873704767
:105C40000C020020034BA0229B691A701A78A02A2C
:105C5000FCD070470C020020034BC2B29B691A7043
:105C60001A788242FCD070470C020020014B5B6A1C
:105C7000187070470C020020024B5B6A1878C0B2A3
:105C80007047C0460C020020014B1B681888704703
:105C90001C0E002008B5FFF795FE024B0022DA60CB
:105CA00008BDC0461C05002070B5074B074CDA6BD9
:105CB000E668011C9579586C2A1C8019751903F047
:105CC000BBFCE56070BDC0460C0200201C05002036
:105CD00073B56C46E271194A0734556D2E788642C9
:105CE0002AD1FF2028701366131C94331B68207878
:105CF0009B6880009165D4651871114B06980C78EB
:105D000018608878536B60430C794979001949060B
:105D1000490E414319609169A0230B70516DD369FD
:105D20000A78FF2A02D11A78002AF9D00A78FF2AC5
:105D300002D11A780A2AF3D073BDC0460C020020A3
:105D40001C05002070B5144C636B1D79EDB2012D5C
:105D500021D1854058781E78000230439E78360461
:105D60003043DE7836063043284214D0FF201871C5
:105D70000A48A16302608C780D78C9786C434906A3
:105D8000490E074A6143506B926901607721117097
:105D90001A79FF2AFCD070BD8C0200201C0500205F
:105DA0000C020020014BDB6B187870478C0200203E
:105DB000014BDB6B187070478C020020014BDB6BD2
:105DC000587870478C020020014BDB6B587070478D
:105DD0008C020020014BDB6B987870478C0200200E
:105DE000014BDB6B987070478C020020014BDB6B22
:105DF000D87870478C020020014BDB6BD87070475D
:105E00008C020020002303600B601B4BF7B59A4205
:105E100030DC1312194C122B1BD89B00E418646E53
:105E2000002C27D0E368013B5D1C23D0D5B201953F
:105E300065681E1CEF5C019D013BED1BF4D42768D7
:105E4000B300DB59002B15D05B190360A3689B5D81
:105E50000EE0A36B266B013B0CD35D00755B551BFD
:105E6000F9D4E66A9B00F25852190260626BD3586B
:105E70005D1B0D60F7BDC046FFEF00000C02002067
:105E8000C02208B5D2000B4B904206D19B691A780C
:105E9000052A0DD005221A700AE01B6C84221B789B
:105EA00092005B065B0E9B18984201D1FFF764FDE0
:105EB00008BDC0460C02002038B5051C1C1C181C6F
:105EC0008D4209DB0498954206DAC01A6D1A6843C0
:105ED000511A03F031FB201838BD044A033013680F
:105EE0008010800018181060181C7047280E0020C1
:105EF000F8B501254E1E6C00B54202DA165FB042BD
:105F00000CDAA61E1D5F115F9B5F401AEB1A584307
:105F1000935FC91A03F010FB4019F8BD0135E9E79A
:105F2000014B18607047C046380E0020014B1868BE
:105F30007047C046380E0020014B18607047C046BD
:105F4000300E0020014B18687047C046300E00200C
:105F5000014B18607047C046340E0020014B186892
:105F60007047C046340E0020014B18687047C04689
:105F7000D8030020F0B5394F8BB0754603950E1C41
:105F8000051C7146381C002401920293FEF778FA32
:105F90006A464F239482201C137504A9221C049482
:105FA000FFF7D0FE2E4B201C1A685368013B10D31C
:105FB000990074581168A4464C1EF7D3976879432A
:105FC00059180131890049596746C91B4018211CDD
:105FD000F2E7D16803F0B0FA224B071C1C68224E8E
:105FE0006588002D03D1336840229A600CE0A188B7
:105FF0003268681A8001791A009203F09DFA6E28BF
:1060000000DD6E20009B9860A37964225343019ABF
:106010005343029A13412278002A04D0124A12688C
:10602000926853439B11326806A9D36001230B7019
:1060300002234B708B707C235B420020CB7008AA3C
:106040005023888008950B710997FFF77BFE034862
:106050000399FEF72DFA0BB0F0BDC046155F0000A6
:10606000D4030020300E0020D8030020F0B5754680
:1060700087B00395274D0291041C7146281C171CFC
:106080001E1CFEF7FDF9244BFA691B68DB799A4068
:10609000131E00DC0123214A311C1268D0685843CA
:1060A00003F04AFA1E4B00901D682F68BC463A1C4C
:1060B0006B68561E16D3191C7143C91889006118E4
:1060C0000439013B0CD3AF6802985743DF190137FD
:1060D0007F00385E009F47430868C01B0860EFE7F9
:1060E000321CE5E76946DBB24B748B746023624671
:1060F00004200B7510234B750A74C874221C04A964
:10610000FFF720FE03480399FEF7D2F9012007B0FC
:10611000F0BDC0460D600000300E0020D803002006
:10612000D4030020F0B51D4D85B0744601940E1CBB
:10613000041C7146281C171CFEF7A2F9184B391CC9
:106140001B68D86803F0F8F9164B00901B681969B2
:106150008A00A2180B1C043A013B07D35F00F05FD2
:10616000009F47431068C01B1060F4E76A46612334
:106170000126C9B20420137310235373167251728F
:106180009172D07202A9221CFFF7DCFD281C019934
:10619000FEF78EF9301C05B0F0BDC046C5600000AA
:1061A000D8030020D4030020F0B5244C85B07546F8
:1061B000019500911D1C7146071C201C161CFEF742
:1061C0005FF96878B37871784000013098404900F1
:1061D000AB7801319940800303F0AEF900226946A3
:1061E000B4238A81051C0B73101C02A90292FFF7CD
:1061F000A9FD134B201C1E683268013A0DD3736849
:10620000191C5143C918890079180439013BF4D38A
:106210000C68A40B6C430C60F7E73369009C9A0090
:10622000A218043A013B04D31468A10B694311601E
:10623000F7E70199FEF73CF905B0F0BD49610000B0
:10624000D4030020F0B589B07446069002912B4823
:10625000714607940392FEF713F9294B1E68294BE8
:1062600034681B6800940493274B1B680593274BE5
:106270001F68009C013C00941FD374680099244A55
:106280006143A5186D18069BAD0001915D19013C95
:10629000EFD30399286803F001F904990B78002BD8
:1062A00007D0059A019953181B5DBA6858435043AB
:1062B000001300042860043DE9E7124B34691E68AE
:1062C000114B1F68013C13D30299A500485903994B
:1062D00003F0E4F83378002B06D0F0223B1992004B
:1062E0009B181B7858438011029B00045851E9E722
:1062F00002480799FEF7DCF809B0F0BDE56100003F
:10630000D4030020300E0020340E0020D8030020DB
:10631000FFFFFF3FF0B51A4C071C0E1C85B07146FD
:10632000201C7546FEF7ACF8164B2A371B683A78E6
:10633000997C4A43316892098A4200DA0A1C997BA7
:106340004A43921101921B7B9A4200DA019302A9FF
:1063500000228A8001220A704A708A707C2252428E
:10636000CA701F220A71062001AAFFF7EBFC201C4D
:10637000291C019EFEF79CF8301C05B0F0BDC046FC
:10638000B5620000300E0020F0B599B0754611904E
:106390000C1CA548714612930B921395FEF770F8EA
:1063A000FAF72CFDFAF736FDA04B1B68F0331B788B
:1063B000002B07D19E4B1B681E7A09960A201F5E90
:1063C000089706E09B4B1B689D7809950427DE5FC4
:1063D0000896994E0025336815A81A68058051273C
:1063E000586814A96F440A7038709A685221532073
:1063F0006944042368440A70037015A951230B7083
:1064000001320B9B92009A1814A90220FFF79AFC04
:10641000A31DDD770233DD777F27631DDF773168CA
:10642000E31DDF774B680A68013BDBB20D93804BBD
:10643000824F1E68824B013A1B6852B20E93814B09
:10644000B4461B6807970F9380231B060693059598
:106450000395002A00DAA3E00D98550043B20A958F
:10646000002B00DA9AE08E68551C75430135ED1853
:10647000A8000B9F0095129D9E00C059AE59069F23
:10648000861BB74200DA0696079DB54200DD0796E7
:10649000664637784E68002F09D0351C55430E9F4D
:1064A000FF187F5D0F9D7843AD6868430013564326
:1064B0001E9F9E19B600F659119F360C301A009E89
:1064C0007500E8536646002854DB0F257557A8422F
:1064D00012DB2768451B7D1925606569102701358A
:1064E0006561F757F67B656876B2B84201DC861BBA
:1064F00000E0BE1BAE196660E568A84204DDDEB2AE
:10650000D7B210960C97E0606646357BA8421BDB3D
:10651000251C08351F26AE579E4200DAEB77E51D95
:106520001F26AE579E4200DDEB77A51D1F26AE57F6
:10653000964200DAEA77651D1F26AE57964200DDC7
:10654000EA77059F0137059785B2209F5E00019588
:10655000BD5B019F7D192F1C209DAF531F9D0A9E7F
:10656000AF5B019EF5191F9F0A9EBD53039F3F1805
:10657000039711E011257557A84206DCA768451B53
:106580007D19A560A5690135A5612569A84200DAD4
:106590002061039E361A0396013B61E7013A58E7F2
:1065A000254B03981B680125D96802F0C5FF7C23A1
:1065B00016A95B42221CCB70E06176231C320026B8
:1065C000281C8E800D700B714D708D70FFF7BAFB1B
:1065D000059FA21D27621F21631D51561F229A5637
:1065E000184B1B68914201DB1D7100E01E71069D76
:1065F000079EE562109F0C9D231C283326631F70A5
:106600005D70E668099F0125BE4205DA2369089C92
:10661000DD0FE2179C42554103481399FDF748FFEF
:10662000E8B219B0F0BDC046296300004000002068
:10663000300E0020380E0020D4030020FFFFFF7F23
:10664000340E0020D8030020F0B589B075460C1C2C
:1066500003907146444804936E4605950027151C27
:10666000FDF70EFFFAF7CAFBFAF7D4FBFCF736FE8C
:106670000123B78333763D4E6A46306806A9037C12
:106680000220537693760423D3765A2313772A1C59
:10669000FFF758FB231C2A331F7080231B066363FC
:1066A000334BA36333681A69324B1968324B1E6847
:1066B000324BB4461B680193013A44D3049F9600C1
:1066C000BF59A859C31B676B9F4200DA6363A76B6E
:1066D0009F4200DDA3630B78002B07D06746BB18F1
:1066E000F027BF00DB191B78584380110E9FBB5960
:1066F0001B0C1B1A11D4487B834202DB019E012034
:1067000030710F200856834212DB2768181A381898
:1067100020606069013060610AE011200856834200
:1067200006DCA668181A3018A060A0690130A061C4
:10673000039F50003B52201C2A300678B34200DAF7
:10674000331C0370B8E70B4B2A341B6822781B7A82
:1067500000209A424041C4B205990348FDF7A8FEC3
:10676000201C09B0F0BDC046E9650000D40300203C
:10677000FFFFFF7F300E0020340E0020D8030020E2
:10678000F0B585B003931A4B00901C680291256800
:1067900001926F1E1BD3636800981E1C7E43F6187F
:1067A000B6008619043E013B0FD3A168012269435C
:1067B0008C469C449444604601998000425830685D
:1067C0009446844461463160ECE73D1CE1E7226970
:1067D000039D029C9300E118E8180023043B013A52
:1067E00004D3CE58C5587419CC50F7E705B0F0BDA6
:1067F000D4030020F0B574468FB0079403900C1CAE
:106800006448714606926D46FDF73AFE0023AB845C
:10681000614D08AE2B6821205F6999699A6822232F
:106820006B4437701A7023260132684404236E4487
:106830009200017033700220A02308A909AFA218AA
:106840003B70FFF77FFA286841698C4683694F1EC9
:1068500002972ED3029A66465A435E430192039DE5
:10686000F2187600019F76425200AA180596069DFE
:10687000019EBF00ED19760004950196023A013B96
:1068800015D38668049F4E439E199D0001367D599D
:10689000B6003659059F2D0CAD1BBE18019FF55350
:1068A000EE17AD1975401688AD191580E6E7029907
:1068B000CCE70AA9DBB262464B708B707E230132B3
:1068C0005B420A70CB700026A1230120039A8E80C0
:1068D0000B71FFF737FA314B2F4C1A682168304B98
:1068E00088691D681660AC46031CFF25013B13D365
:1068F0004C69039F4443E41864003C5F67463F785B
:10690000BC42F3DB9E4200DADEB29D4200DDDDB226
:1069100017683C191460E9E70CA901240423CB7023
:1069200000276423201C8F800C700B714C708C70BE
:10693000FFF708FA194B1A68194B12681B685B7845
:106940009A4220D9144F69B23B68039F9A695B69E8
:106950005A4373B25B1AD90FCB182341EB18AD1809
:10696000A540DBB2E95F9B18039DA340EB5E271CAB
:10697000994208DDB218039EA240925FD917D70F43
:1069800093424F41FFB203480799FDF791FD381C30
:106990000FB0F0BD95670000D4030020D80300209D
:1069A000380E0020F0B58BB0744603900E1C3348AF
:1069B000714607940292FDF763FD314B1D68314B20
:1069C00028681C68A769391C02F068FD2E4B1B68FB
:1069D000DB799840002800DC0120EB6802995843DD
:1069E00002F0AAFD6169BB005B424A1E8446381C66
:1069F000029350437B005C425343C019039D8000C7
:106A0000F31804942818059300910024009D013D7B
:106A1000009515D3059E021CA61906963B1C043A48
:106A2000013B08D3069E5D00765F65467543166898
:106A3000761B1660F3E7029A049B8018E418E5E7DA
:106A400021242225FBB208AA6C446D4411702370E6
:106A50002B7009AA6023232625240420137008A97B
:106A60001023039A6E446C4430702370FFF76AF968
:106A700002480799FDF71CFD0BB0F0BD4569000009
:106A8000D8030020D4030020300E0020014B1860F2
:106A90007047C046400E0020014B18687047C04642
:106AA000400E0020014B18607047C0463C0E00208D
:106AB000014B18687047C0463C0E0020014B186817
:106AC0007047C046DC030020F0B5724687B07146BF
:106AD0005F480592FDF7D4FC5E4C002120680A2235
:106AE000343002F0EBFD206800210A223E3002F033
:106AF000E5FD206800212822483002F0DFFD2068F3
:106B000000210A22703002F0D9FD206800210C22F9
:106B10007A3002F0D3FD206800210C22863002F08A
:106B2000CDFD206800210522923002F0C7FD2068CB
:106B300005220021973002F0C1FD474B25681E68F1
:106B4000F369346A5B00181B61000002019302F0D4
:106B5000F3FC0490A860B06A726A00905200009B37
:106B6000101A59000002029202F0E6FC19235B425F
:106B70002B613A4B0390E860686101981F684142BD
:106B800002987B1DDA7F4042331CD633019018886F
:106B900060434018002A0ED039680139614302F081
:106BA000CBFC331CD833041C009A1888019B50433B
:106BB0007968C0180DE079680139614302F0BCFCC6
:106BC000331CD833041C009A1888019B5043396841
:106BD000C0180139514302F0AFFC844200DA041CB2
:106BE000E3179B0F1C197968A4102C6204983C6869
:106BF0000139039A43000902013C59182402530049
:106C00001C19A961EC610537FB7F371CD83600964B
:106C10002E1CD637AC36B035002B07D0009B188819
:106C2000000402F089FC3060388806E038880004EF
:106C300002F082FC009A30601088211C000402F0EF
:106C40007BFC059928600248FDF732FC07B0F0BDD7
:106C5000696A0000DC030020400E0020D4030020FD
:106C6000F8B5134C7146061C201C7546FDF708FC50
:106C7000104B00211A68201C131C7A3319700E4B1C
:106C80001B681B7C013BDBB2FF2B0DD059008F5BD7
:106C9000191C3C3149003CB25118002C01DD8F8099
:106CA000F0E700248C80EDE7291CFDF701FCF8BD1E
:106CB000016C0000DC030020D4030020F0B5744612
:106CC00085B002940E1C041C71461F48151CFDF76C
:106CD000D7FB1E4B1B681A6AD2B2013AD2B2FF2A06
:106CE0002AD0F7685300FF5E696860680191002F41
:106CF0001AD0E768FF5E002F16D0C05A716807B23D
:106D00000397C95E039F7F1A7F10BC4601996044B8
:106D1000A768C852F95AB76808B28446F85E674651
:106D2000381A4010411804E00199C05AA768C852A7
:106D3000F95AA868C152D0E7237803482B7002990A
:106D4000FDF7B6FB05B0F0BD5D6C0000D40300207C
:106D5000F7B575460195144D041C0F1C281C71468F
:106D6000FDF78EFB114E0A2230680021703002F0D0
:106D7000A5FC0F4B36681B68281C1A6AD2B2013A70
:106D8000D2B20023FF2A09D0E56851004B53B11855
:106D90000D1C303538312B718B71F0E72370019960
:106DA0003B70FDF785FBF7BDF16C0000DC030020B4
:106DB000D4030020F7B5124E73467146301C019380
:106DC000FDF75EFB0F4D002428680527031C7A336E
:106DD0001C703A1C211C923002F070FC28683A1C8E
:106DE000211C973002F06AFC2868211C0A227C30A2
:106DF00002F064FC301C0199FDF75AFBF7BDC04658
:106E0000556D0000DC030020F8B5154E041C0D1C68
:106E1000301C71467746FDF733FB124B301C1B6864
:106E20005A1DD17F9A1D00290CD021882E882680DA
:106E30002980D27F002A0ED01A680733DB7F013AFF
:106E4000D31A04E0D27F002A05D05B68013B228878
:106E50001B029B1A2380391CFDF72AFBF8BDC04694
:106E6000A96D0000D4030020F0B5714689B07646C4
:106E7000071C41480596FDF703FB38687A6807ACA4
:106E800069461E312080201C0A80FFF7BDFF3B4B66
:106E90001B685A1DD17FDD1D394A41CB00290ED018
:106EA000EB7F411E013EC91A3602090203961268A1
:106EB000002B0ED01669DB019B19566910E0711E7C
:106EC000EE7F0138801B0002090203901268002E39
:106ED00002D19368D66803E013695269F601B618C7
:106EE000284A1568286801900022A05E019AC018FF
:106EF0005B00C918504302F01FFB80B20490208051
:106F00006868694602901E20085E029A039B8019F9
:106F100076009919504302F00FFB6E4680B22B1C8D
:106F2000F083D433049E1B7832B29A4206DD019E70
:106F3000F11A8A4203DB321C013AD31A23802B1C3C
:106F4000D5331B7800B2984206DD029EF21A9042B9
:106F500004DB321C013AD31A6846C38307AB002115
:106F60005B5E6A463B601E23D35E03487B600599E7
:106F7000FDF79EFA09B0F0BD096E0000D4030020B1
:106F8000DC030020400E0020F0B572468BB0714645
:106F9000041C5E480592FDF773FA5D4B00211B68E7
:106FA00002915A681D6A013A120203921A68013D61
:106FB000013A1202AB0004926E000193691C00D1E9
:106FC0008DE0544B1B681A1CE6321778012F15D13F
:106FD0002269EA33905B19780022A36988420CD9B0
:106FE0005F556B469A836946B5230B770E2006A939
:106FF0000692FEF7A7FE029700E05A55454B1F6820
:107000003B1CEB331B78012B63D1E3689A5F3B1C7D
:10701000EE331B889A425CDD61688A5FFF2A09DDD6
:10702000A1688B5FFF2B05DD03998A4202DC049A7D
:1070300093424EDA364B62691B680533D97F364B73
:10704000002915D0019918685218002301215156C2
:10705000D356CB1A011CB03109681B024B430321E4
:10706000515692781B1452B2891A0902AC3014E0BE
:10707000019918685218022303215156D356CB1A8E
:10708000011CAC3109681B024B4301215156127897
:107090001B1452B2891A0902B03002680A20514307
:1070A00009148B4201DB584301E04843191C02F0EC
:1070B00043FAEC373B7898420BDDA2690123535524
:1070C00008A90022B6230E208A8008920B71FEF7D1
:1070D00039FE019B013D043B023E01936EE7029A9B
:1070E000002A05D109480599FDF7E2F90BB0F0BD7A
:1070F000074B1B681B6A013BF4D3E1685A00525EE0
:10710000002AF8DDA1690122CA54F4E7296F0000C2
:10711000D4030020400E0020DC030020F0B57246AE
:1071200093B07146041C59480392FDF7A9F9584AD7
:10713000584B12681B6811793822514359182C3169
:1071400004A802F079FA544B00261B685A681F689D
:10715000013A120202920733DB7F013FFF1A3F021E
:107160004D4B1B681A6A964200DB88E0E1687500A7
:107170004A5F002A00DC80E0454A12681279012A41
:107180007BD06268505FFF2819DC0533DB7F0499F0
:1071900005AA002B02D06B46323301E06B461E334A
:1071A000FEF7A6FE616800B24B1900215A5E013A53
:1071B000FF3A504380110130FF30188020E0029ADE
:1071C000101AFF281CDC0533DB7F049905AA002B6D
:1071D00001D00FAB00E00AABFEF78AFE029A6168AD
:1071E000013AFF3A4B1901920022995E029A00B2CD
:1071F000511A0139FF394843019A8011121A1A8035
:10720000A368585F244BFF2819DC1B6804990533D9
:10721000DB7F05AA002B01D00AAB01E06B463233BD
:10722000FEF766FEA16800B24D190022AB5E013B7D
:10723000FF3B584380110130FF3028801DE0381A91
:10724000FF281ADC1B6804990533DB7F05AA002B95
:1072500002D06B461E3300E00FABFEF749FEA36879
:1072600000B25D1900216A5E7B1EBA1A013AFF3A2C
:107270005043FF3B80111B1A2B80013670E70348F7
:107280000399FDF715F913B0F0BDC046BD700000BD
:10729000DC030020400E0020D4030020F0B5764629
:1072A0008FB0041C0F1CC14871460796FDF7E8F823
:1072B000BF4B1B689E680696DE6802961E690196A3
:1072C0005E699B6905960393FEF7E4FCB94B0126C2
:1072D0001B68E4331B780496002B54D000260496D8
:1072E000B54B1B681B6A9E424DDA78687500435F98
:1072F000B9680A934B5F0AA80B93FFF7B5FDE268E4
:10730000535F002B3DDD6068A168435F08A80893C8
:107310004B5F0993FFF7A8FD089B069A9A4209DA8A
:107320000298984206DD099A0199914202DA05987D
:10733000904221DCF9684A5F002A19DD9F4A1268F1
:1073400092193032127952B2012A11DD069803994E
:10735000421A9A420CDA029842189A4208DD0198C1
:10736000099B421A9A4203DA059842189A4206DCAF
:10737000E16800234B5304E00122049201E0012361
:1073800004930136ACE701268B4B03961B68039EE2
:10739000186A013E0196864200DBC8E0039E8848D9
:1073A000796835186D004B5FBA680A93535F0AA875
:1073B0000B93FFF759FDE668735F002B00DC86E056
:1073C0006068A168435F08A808934B5F0993FFF7C3
:1073D0004BFD0A9B099E9C46784B02961B68019EBA
:1073E00006939B1970331E78764B089A0B981B688E
:1073F000002E01D1503300E05133F9681B784E5F05
:10740000002E0DDD029E301AC117401848409842E8
:1074100006DA6646911BC81709184140994273DB8A
:10742000049E002E70D00CAE317880235B420B435B
:10743000DF210B4040210B433370A169019BC85CE5
:10744000012331781840102399438C4603990F2368
:10745000194005910001614608430599984301438D
:1074600010121840317071780590029899438C463B
:1074700001120901059800916146084300991840DE
:10748000B270029AE36801437170F2705A5B131C88
:1074900012B2FF2A00DDFF233371069B301CA83394
:1074A0001B6801999847301CFEF7FEFBFE68434BB2
:1074B000725F1B68019E9B19002A03DD1A1C703243
:1074C000012302E01A1C7032002313701CE0F868DC
:1074D000435F002B18DD0CA800234360039B0F21A2
:1074E0000B40402213430A9A037013129C460B9BD5
:1074F00082701E123601019666463140019EC370AD
:107500000E434670FEF7D0FBE068F968435B6268A3
:107510004B53535B7E68A0687353435BB968226921
:107520004B533E69535B7353039E01362CE71B6933
:107530005E1E03960F2603981E40204D013043D057
:107540000398296840000B181A1C8832019000200B
:10755000125E7C33002A0FDC1B881AB2002A16DD6B
:1075600000210CA80C914160802131430170FF2A59
:1075700000DDFF23037108E000215B5E002B06DCC9
:107580000CA800230C9343600670FEF78DFB019A54
:107590002B68013E9B181A1C7C331B888832138091
:1075A000039B013B03930F23C5E7C0463D720000D8
:1075B000400E002040000020D4030020DC03002007
:1075C000FFFFFF7F3C0E002023783B702B681A1CC6
:1075D0007A321178117338780122002802D10A1CFE
:1075E000511E8A419E331A70FEF7A4F9024807998A
:1075F000FCF75EFF0FB0F0BD3D72000010B5022435
:107600008B7804575AB2944200DD8370CB78032400
:1076100004575AB2944200DAC3700B78002404571E
:107620005AB2944200DD03704B78012141565AB2A0
:10763000914200DA437010BDF0B58FB00A910A9CF8
:107640000893C36864001D5F0C940695540004946D
:10765000069E1C5F0A9D43683619AD0005960131F0
:10766000960009955D19071C0D91985906992B688C
:1076700060434B430599C0180B9201F05DFFBB6856
:1076800000B22860099A98599D182B6844430698BF
:1076900005994343E01801F04FFF3969099C00B296
:1076A000286004220819089901F0C6FFFB680C9DA8
:1076B000049C5A191B19108819884118118000223E
:1076C0001A807B695A191B5B0025505F19B28842EA
:1076D0000ADA1380BB69049D1A190C9C52781B1995
:1076E0005A70BB695A5D1A550B9B013301240F2B4D
:1076F00009DC159D0998A9592A1815689C400C4069
:107700002C431460F1E7159D0023AB510A9D0B9E9D
:10771000211CB140AC40159AA446CD430B9EB34208
:107720001ADA1068014214D00A9EB34203DA6446A2
:10773000204310600AE00A9EB34207DD159C099EB3
:10774000A019046801269E40264306601068284060
:10775000106001330432E1E7089C247864B2079496
:10776000089D0123EB56079E9E4200DDACE0089D7C
:10777000AD786DB2089E04950323079AF356049CD6
:1077800001329C4200DD9DE0624B049C1B68149D0D
:107790009E68724301321219AA181178B446013951
:1077A000112900DC8BE00120052340420024013B2D
:1077B000002B29D0584EF51801267642AE57079D6A
:1077C000AE19013665467543534E0595F518ED79AA
:1077D000049E6DB20295149DAD19059EAD19029ED1
:1077E000AD1905956D78013D0F2DE0D80A9EB54283
:1077F00002D00B9EB542DAD1461C03D0A842D6D0A7
:107800000124D4E7281CD2E7002C58D0122955D1E6
:107810000D9C052514700695069C013C0694002CD1
:107820004DD03D4B069E07249A19131C013B1B7833
:10783000079E5BB2F618374B14571A68331C9268D0
:1078400001335343049D01332C19149D1B19EA186D
:107850001178B4460029DFD1169E5B009B5B002B9C
:10786000DAD0122111707868099D4619F8680C9DCC
:107870003268401902900088099D019001B2181CDD
:1078800060434A4300021018BA68541965462268DA
:107890005D4351432D02AC46614405910199029A22
:1078A0005D18ADB215802DB2291C01F045FE291CD2
:1078B0003060059801F040FE2060ADE71170049D36
:1078C000013557E707924BE70022AA56089E01238D
:1078D000F3569A421BDC089C0223E356089D0320C2
:1078E0002856511C834210DC0A48149D00680B9EE8
:1078F000806841430131C918691808780138B042DD
:1079000001D10D9C0C700133E8E70A1CDEE70FB0D3
:10791000F0BDC046D403002010970000F0B591B030
:1079200075460B91061C714641480D950C920793C4
:10793000FCF7A6FD0024F7686300FA5E002A6DD00C
:10794000B0690125C3185D571B7809955BB2089390
:10795000013D0695099F069D01370A97BD425DDCF2
:10796000089F013F0597089B059F01339F4252DC0A
:10797000304B06991B6801319A68059D51430B9F56
:10798000481C40193D5C013D0F2D40D8AC423ED013
:1079900077696300DB5F284F40003F683F89BC4642
:1079A000079FC05B834232DC089F6046C91943438E
:1079B0000131079F4900C95B9B118B4227DA0A9F5F
:1079C0007A43059FBA180132079F5200D25B934257
:1079D0001DDAA54202DB2B1C251C1C1C3769A100EB
:1079E000791804220FA801F027FEA90079180FA822
:1079F000FFF704FE0B9F221C00970C9F301C019781
:107A0000079F291C02970FABFFF716FE2C1C059D44
:107A100002350595A7E7069D02359AE701340F2C3C
:107A200089DD03480D99FCF743FD11B0F0BDC04658
:107A3000BD780000D40300203C0E0020F0B5A7B0B4
:107A40007546071C0C91C848714613920D931A9500
:107A5000FCF716FD139A0D9B381C0C99FFF75EFF7F
:107A60002C9EC24B3278012A07D13A78012A04D9D8
:107A70001B689C881494DB8803E01B681D881495A0
:107A80005B880F2615930696069B069C013B002CEF
:107A900000D171E1139C9A00069D12590795EA40A6
:107AA0000F9206930F9D002DEED0079E102EEBD067
:107AB0000F9E0120064200D14FE1079D069C7B6886
:107AC000A400AE001959BA689B590894C91A1459F0
:107AD0009359CD17E31A4C196C40DD1710945C19BB
:107AE0006C40109D0B94A54202DD1190180203E03A
:107AF000002408021194191C01F01EFD3C691CAD04
:107B0000A11904221290281C01F096FD0898211852
:107B1000281CFFF773FD7968089CFB680859079CCF
:107B200020906100CC5E09947C68A4590A94069C5C
:107B30006200D45E099B099A58430A9BA2186343CA
:107B4000111CC0180E9201F0F7FC21900A98BB6836
:107B5000089922905858099A23909E59504374438B
:107B60000E99001901F0E8FC0024249000211DA8C2
:107B70000C22259601F0A2FD2C5701260994AE5740
:107B8000022416962C577A4B1794ED781B686DB229
:107B900018951993099C169DAC4200DD9FE0099D44
:107BA000179E2D020E9508960999089D189E013181
:107BB000B54200DD91E0199C089EA0680C9C4143F1
:107BC00001318919645C8446231C013B0A940F2B04
:107BD00044DD0020012205235242041C013B002BFE
:107BE0002BD0644EF51801267642AE57099DAE198A
:107BF0000136654675435F4E0595F518ED79089E8B
:107C00006DB204950C9DAD19059EAD19049EAD197C
:107C10001B956D78013D0F2DE0D8069EB54202D030
:107C2000079EB54205D1561C05D0AA42D6D00124E4
:107C3000D4E70120D2E72A1CD0E7013249D049001D
:107C4000002C01D1002802D10D9C605A11E00D9D3D
:107C5000685A0A99113901F06FFC0AE05E1C38D0AD
:107C6000069CA34202D0079DAB4232D10D9E490033
:107C7000885B00282DD0089C03232102013B28D3D8
:107C8000119D20AC23AA9E00002D09D095590E9A73
:107C9000551B129A5543A2592D12551B6D1A08E017
:107CA000A559129C4D1B654392592D120E9E551BD2
:107CB000AD1BEA17AD185540FF2DDFDC802676009E
:107CC000751B45439C001DAAA6582D127519A55079
:107CD000D4E7089C0134089466E709915AE71F9B92
:107CE0001D9C9C4200DD1C1C119E002E06D10B9D8C
:107CF000331C002D0DD0109E10950B960B9D1099E6
:107D0000A80101F019FC3F2800DD3F20194B18188D
:107D1000037C2D21149E159DC81A70436B43C01817
:107D200001F00AFC44431E9BA412A34215DD079EEA
:107D3000069CA64201DB079406960C9D139E0D9CA3
:107D400000951CAB01960294381C0799069AFFF720
:107D500073FC069B079D07930695079E0F9C0136B3
:107D6000640807960F949DE6DD7900003C0E002024
:107D7000D4030020109700002C4B3C7018680121A0
:107D800024304942102201F099FC069C251CF86819
:107D90006600825FE3B2002A25DD3A7801323A704C
:107DA000224A126812190532D5779D4219D07A6895
:107DB000A300D158A8001150BA680790D1581150AB
:107DC000FA686800925B011C101CFA6888523969D5
:107DD000079A8818C918042201F02EFCF8680023BD
:107DE00083530135EDB20134102CD0D123A90023E7
:107DF00023938B800E4B7F201B680C9D1A680A70A2
:107E00005C684C709A68CB788A7083430120034386
:107E10001218CB70AA18302306200B71FDF792FFC1
:107E200004481A99FCF744FB27B0F0BDDC0300209E
:107E3000D4030020DD790000164BC2171B688018A0
:107E400050401A1CAC3270B5B0331468CA17891888
:107E50001D68514044434D4324142D14AC4202DBB1
:107E6000231C2C1C1D1CA001291C01F065FB0A4EC3
:107E70003018037C281C002B0BD05A22D21A523601
:107E80005200955B5B0068439D5B00146C432414B7
:107E9000001970BDDC03002010970000F0B5754696
:107EA0009BB0041C0F1C844871460D9508921E1C43
:107EB000FCF7E6FA814B1D6823782A6A934200DDBD
:107EC000131C01213B70494210220EA801F0F6FB61
:107ED00012A8FF21202201F0F1FB794B2D6A1B68CB
:107EE00009950A93774B00251B6804950B93049D15
:107EF0000998854257DA0898049DC0686D00435F71
:107F00000795002B4AD0049B0A9D12339B000B98C7
:107F10005B592578C0681B010C9500251B18059539
:107F2000012506936D4205980C99C3B28B421FD26E
:107F30000598E16843005B5E002B15D0830007992C
:107F40007068425E6168C8580799801AB268525ECC
:107F50009446A268D1586346C91AFFF76DFF069987
:107F6000884201DA059D0690059A01320592DAE70A
:107F70006A1C13D00EAB59576A0012AB013108D0FE
:107F8000995A0698814209D99852049B0EAA5355D2
:107F900004E006980EA99852049A4A55049B0133AE
:107FA000DBB20493A3E700252378AB4228D90EA9BE
:107FB0004E5D73B2013320D06068A9004258F6B21A
:107FC00078687300C252A0684258B868C252E0682C
:107FD0006A00105A0492FA68D0527A692369B00094
:107FE00010185918042201F027FB354B049812AAE7
:107FF0001B681236825AB600F2500135EDB2D3E753
:1080000000252378AB423ED90EA94B57013337D117
:10801000E3686A009A180026935F0492002B2FD021
:10802000264B00201B681B6A0593059EB04227DA89
:1080300008994300C968CE5E002E1ED1FE68F6186E
:108040000022B15E0696002917D162680EAE705507
:10805000A90056587A688000D652A2685658BA6865
:10806000D652049A069E13887A69338023691018C1
:108070005918042201F0E0FA02E00130C0B2D4E75E
:108080000135EDB2BDE70E4B18680C4B1C680023A0
:10809000C21824321178256AA94202DA0EAE715C48
:1080A00000E0FF2101331170102BF1D102480D992E
:1080B000FCF7FEF91BB0F0BD3D7E0000D4030020AC
:1080C000DC0300203C0E0020F0B57446A3B01394EE
:1080D0000B91041C71468D480C92FCF7D1F9FEF708
:1080E000EDFC8B4D0D90291C08310A2217A801F0D8
:1080F000A3FA291C12311AA80A2201F09DFA854B15
:108100001B681B6A013B0793079E013600D1F6E00E
:10811000079DE6686D00735F0895002B00DCEAE0C0
:10812000079F6069BB00C0187A4B02221B680321BD
:10813000825641561093784B00251B6884460E9159
:10814000119306950A950E9FBA4264DC6646012794
:10815000F7570021100271560F9712900F9E531C73
:10816000B14256DC109E4F1CB568381C68430B9E0C
:10817000C018335C0597102B23DD0523013B002B32
:108180002DD0664EF718F618013E3678FF7976B294
:108190008E1901366E437FB204970B9F0396049E9F
:1081A000BF18BE19039FF7197E78002EE6D0119FE5
:1081B00076B2BE190436F67F079F76B2BE42DDD195
:1081C0000AE0002B0BD00D9E1F25F31804335D57DA
:1081D000079F0023BD4202D10C9D4000435B6668AF
:1081E000089F0902F05F129F0A9EC01BC517401925
:1081F00068405843089DA7683618785F069D411A65
:10820000C817091841404B43ED180A960695059981
:10821000A4E71A1C97E7089D6068A368425FD0171F
:10822000000E801800120002101A5A5FC117D317EF
:108230001B0E9B181B121B02D31ADD1740185B196B
:1082400048406B40802802DD80225200101A802BAB
:1082500002DD80225200D31AC018052117AA1AABDA
:10826000FDF746FE2E4B051C1B68E6683D3319786A
:10827000089F40235B1BF05FA02200930023FDF7C3
:108280001BFE2E18E068C71900217D5E0A98291C84
:108290007043059701F050F9071C0698291C70439C
:1082A00001F04AF9BF118111381CFFF7C5FD1A4BC7
:1082B0001B681B6A984200DA181C2269089D059FFA
:1082C00050530023FB5E15A91F9300238B8020933E
:1082D000219301230B7005234B708B707C2380B29C
:1082E0005B42079E1E90CB701220B0231DAA1D96E4
:1082F0000B71FDF727FD079D013D079504E7034836
:108300001399FCF7D5F823B0F0BDC0466980000092
:1083100010980000D4030020DC0300201097000018
:108320003C0E00200F4AC378126810B551685CB249
:1083300001398C4201DA0133C370837859B20029C4
:1083400001DD013B83704378126859B2013A9142D2
:1083500001DA0133437003785AB2002A01DD013B90
:10836000037010BDD4030020F0B593B0754605919D
:10837000071C7146CD48089209930B95FCF780F8CD
:108380000EA900238B80CA4B059C1B689A6858680D
:108390001E688A70012301324870CB70A21808232E
:1083A00006200B710E70FDF7CDFC1023013BDBB2F4
:1083B000FF2B0BD03D699A00A9187F2008708870A8
:1083C0003E69FF21B2185170D170EFE7B94B00221E
:1083D0001B68189C1A600923E356189D0822AA56A8
:1083E000934269DB189D0B22AA56189C0A216156FC
:1083F0008A425FDBAE49059E0868591C806841438C
:108400000131891870180478251C113D2D2D02D8D2
:10841000002101704CE0013CE4B20F2C48D8099DCA
:108420004900485BA3497E6809680D6801350D6005
:10843000A1007518061C5643B4462E686400B44467
:1084400066462E60BE687518061C5E43B4462E68EC
:10845000B44466462E60FE6835192E8886192E8033
:108460003E6975180226AE57B24200DAAA703E691C
:1084700075180326AE57B24200DDEA703E697518E2
:108480000026AE57B34200DA2B703D69691801250A
:108490004D57AB4200DD4B707E69311900268D5F70
:1084A000854205DA0880B86901194B70B9690A5527
:1084B000013A9AE7013B90E700260496F868049C8D
:1084C000035F002B01D10024F8E0049C3D696400A7
:1084D00028190694FFF726FF3E69331901269E5797
:1084E0003869069C002203199A56964200DAD6E0B3
:1084F000DB785BB202933D69069C2B199B78029D49
:108500005BB29D4200DAC8E0694B029C1B68059D86
:108510009B6801930198731C434301331B19ED18A9
:108520002A780395002A02D03F2A00D0B1E0099DA5
:108530005B005C5B002C00D1ABE000230D930523B6
:10854000013B002B21D05C4A0725D1180A1C4D574E
:10855000012149425156019871180131484305994A
:10856000844602980A185219624451784A1E0F2A0A
:10857000E6D800220DA8855C002D01D18154DFE7EB
:108580008D42FBD00132D2B2F4E70DAA9A5CDDB283
:108590000195002A04D00133042BF6D1019302E0A7
:1085A000019D002D75D00199201C00F0C5FF019D93
:1085B000039911350D700795029D311C45434143C8
:1085C00003950A91002301997D688C460121494257
:1085D0008C440DAA63451CDAD25C241A013A91003E
:1085E0006D1800922A6801339446039A94446246B7
:1085F0002A60BD6869180A6894460A9A94446546D8
:108600000D600099FD684A00AA18118809181180A8
:10861000D9E7D35C5B1802999A006143AD182868CA
:108620005B0041182960B968F8688A18211C7143F9
:108630001568C318691811601A88079914191C80E5
:108640000023122925D0634523DA01331A1C019D2A
:10865000AA42F8DA0DA8C11801390978105C01396D
:108660000138C9B2C0B20124814208D2089D8900F4
:1086700069188440201C0C682043086007E0089DAE
:10868000800028188C40211C0468214301600132BD
:10869000DDE7029C013C02942DE7013E20E7049DAA
:1086A00002350495202D00D008E70CE7098300006F
:1086B000D4030020DC03002010970000FE68620055
:1086C000925BE3B2002A19D07868A500461911B26E
:1086D00032680291100200F02FFFBB6830605E1913
:1086E000316801340802029900F026FF3A693060CF
:1086F0005019FFF717FE102CE0D1231C10A93B7076
:1087000000238B800B4B059E1B6806209A681C6813
:108710005D688A7001230132CB70B2182D230B7172
:108720000C704D70FDF70EFB03480B99FBF7C0FE74
:1087300013B0F0BDD403002009830000F0B57746E4
:1087400087B0051C0E1C704871460597FBF798FE14
:10875000F8F76CFB6D4B071C1B68287A697A01904F
:108760001C68FA20800003914843211C00F0E4FEBD
:108770003A6900901778002F16D0012F16D1644B5C
:108780001B681B6A013B0DD3D7685900795E00292D
:10879000F8DD604F3F68E0373F88BC460127614500
:1087A00007DB04E0012704E0012301E001273B1C73
:1087B0005B42516892685800095A125A0291049219
:1087C000022E17D004D8002E0AD0012E0DD08FE033
:1087D000052E30D0062E53D0042E00D088E027E09E
:1087E000002B64DA012F2FD184E0002B68DA012FEF
:1087F00075D17FE0002B03DB019F4F2F60D979E01B
:108800000199FA2080004843211C00F095FE414B5D
:1088100003241B681A1CE2321288904205DCE43300
:108820001B880024984200DA0524012F39D161E029
:10883000012F09D160E0002F08D1364B009A1B6848
:10884000E4331B889A424ADB082456E0002BFBDB0A
:108850002968029F0023CB5E6A6838B2049FC01A61
:108860000023D35E39B2C91AFFF7E6FA294B1B6819
:10887000DE331B789842E7DC00236B7206243CE071
:108880000724002F39D00424002B36DB214B009F16
:108890001B68E4331B889F422FDA6B7A01336B72BB
:1088A0002AE0022C0CD0052C19D0012C25D12868E7
:1088B000029F01240780049F686807802C721CE0D7
:1088C000019F28687B00029F02241F522B7A049F7D
:1088D00068685B001F522B7A01332B720DE0013E5A
:1088E0000023012E01D9039B01336B72052404E0A0
:1088F000002402E0042400E0341C03480599FBF73F
:10890000D7FD201C07B0F0BDDD8600004000002030
:10891000D4030020400E0020F0B52C4D85B07446E5
:108920000394071C0C1C281C7146161CFBF7A8FDA1
:108930000422A35E0622A05E0025C01A64235843C9
:108940000223E15E0022A35EC91A00F0F5FD762342
:10895000021C1A3AFF3301909A4230D80295002245
:10896000BB5E64205843019900F0E6FD029B81B292
:108970003980012B0DDDB31E00229B5E0022B05E0C
:1089800009B2C01ABB1E00229B5EC91AFFF754FA37
:108990002D18029B0237013302930236162BDED1CB
:1089A0000422A05E64260199704300F0C5FDA080FA
:1089B0000623E05E0199704300F0BEFDE0800348AD
:1089C0000399FBF775FD281C05B0F0BDB9880000C0
:1089D000F0B52F4F95B07546039501901D1C02917F
:1089E000381C7146141CFBF74BFD0422AE5E0622B8
:1089F000AB5E03219B1B181C009300F09DFD2822F9
:108A0000A35E82190124934200DC002441008E19E8
:108A1000E4B2B34201DD02231C43029E2823F35E2D
:108A20000026AA5F8018834201DD042004438A18CF
:108A3000934201DD08231C4304A80021402200F0DA
:108A40003DFE032305930623079301230893042384
:108A5000099307230B930223109305231193A4007A
:108A600008236A4613931034A358019C009963703D
:108A70000020FFF7E1F91A9D011C0A20684300F06D
:108A80005BFD03992070381CFBF712FD15B0F0BD9B
:108A900071890000F0B5744695B0039402900E1CE5
:108AA0002F4871460024171C0125FBF7E9FC0194AF
:108AB000152D09D10021735E2820325ED21A282399
:108AC000F95E00243B5F07E0019C6B00F15E325FC2
:108AD000019C8A1AF95E3B5FCB1AA821FF315143F2
:108AE000012489128B4200DC00241E48424392126A
:108AF000934201DD022004435242934201DA0422F0
:108B0000144349428B4201DA08231C4300214022CE
:108B100004A800F0D3FD012304930223059303234B
:108B2000079304230B9308230C9307231093062326
:108B30001293A400052313931034029869466258D7
:108B4000019C4319013B023401351A700194162D22
:108B5000AED103480399FBF7ABFC15B0F0BDC0469E
:108B6000358A0000A7090000F8B5104F051C0C1C41
:108B7000381C71467646FBF783FC381C0C4BA5422B
:108B800007DD2C1BA412032C00DD032464001C5BF6
:108B900006E0651BAD12032D00DD03256D005D5B56
:108BA0006419311CFBF784FC201CF8BD098B000004
:108BB0002C980000F0B57546D5B003950091051CC2
:108BC00071464448161C0193FBF75AFC0024012708
:108BD000019B0234013B9F4221DA2B199A1E00218E
:108BE000505E2A5F0321801802229B5E0137C01865
:108BF00000F0A2FC009A102369461B195852131961
:108C00009A1E0021505E00990A5F032180180222FB
:108C10009B5EC01800F090FC2CABE052D8E7019F9F
:108C2000AC1C023F7F0069463A1C201C12310294A2
:108C300000F002FD009C694602343A1CB231201C4F
:108C400000F0FAFC009900220B880092F3800B8858
:108C50000127B3802B8873802B88029D3380019B72
:108C60009F4230DA0023E85EAB1E00215B5E0022EB
:108C7000A15EC01AA31E00229B5EC91AFFF7DCF892
:108C8000009B0222B15E1B1800932B881AB29142FE
:108C900000DA73802B880022B15E1AB2914200DDA7
:108CA000338023880622B15E1AB2914200DAF38043
:108CB00023880422B15E1AB2914200DDB3800137ED
:108CC00002340235CBE703480399FBF7F1FB009828
:108CD00055B0F0BD558B0000F0B5A3B07546141C1F
:108CE00002900391414871460B950A93FBF7C8FB2C
:108CF000201C152100F020FC012406900194002581
:108D000001990A9A91424EDA0199029A4F00D219BA
:108D10000792039A0299BB1ED719C9180897D7184A
:108D2000079B04910020185E089A0023CB5E002167
:108D3000515EC01A0022BB5EC91AFFF77DF8069982
:108D40002B1805908B4229DB049A4D1B0023D25E21
:108D500000217E5E0992089A05990020105E801B12
:108D6000684300F0E9FB079B361809990020185E5C
:108D7000B6B2401A6843059900F0DEFB099D630016
:108D80002818302180B2C9186A46049D885217AA53
:108D90009E52288001343E80002302E0019D01356F
:108DA00001951D1CACE7152C0BD1114C029D13191C
:108DB0005B00EA5A5A21039C69440A80E25A17ABC5
:108DC0005A850298694632312C22023000F034FC78
:108DD000039869462C225E31023000F02DFC0348D6
:108DE0000B99FBF765FB23B0F0BDC046798C000002
:108DF000FFFFFF7FF0B5244F8FB07346051C71460F
:108E0000381C0393FBF73CFB2B7A06AA2868696899
:108E1000FFF7D0FE1D4B021C1B680024DC331B88AF
:108E2000984229DD2B7A28686968FFF755FF2A6880
:108E3000686806A9FFF770FD009006AB05A82968D1
:108E40006A68FFF7C5FD06CD08A8FFF723FE104EA0
:108E50006D463368EC74A03313351B68281C08A9D1
:108E600098472B78041C002B06D1336808A8A4333C
:108E70001B6805A99847041C381C0399FBF718FBCD
:108E8000201C0FB0F0BDC046958D0000400E0020A4
:108E9000DC03002070B5074C061C7146201C75468B
:108EA000FBF7EEFA044B291C201C1E60FBF700FBAD
:108EB00070BDC046358E0000440E002070B5074CD2
:108EC0007146201C7646FBF7DBFA054B201C1D681B
:108ED000311CFBF7EDFA281C70BDC0465D8E00000A
:108EE000440E0020F0B595B009931AAB1B78754677
:108EF0000C900691C5487146109311950A92FBF7A4
:108F0000BFFA069EC24C00237372F37220687F235F
:108F10003372B3720379002B07D1BD4B1B689A7B68
:108F2000002A00D005E107921AE10323C356202747
:108F3000FF1A0223C3567F00FF1A7F10FFB2079764
:108F4000099F7F6805970622815E0823C25E0A2377
:108F5000C356C07A40B20090381CFCF7ADFFAD4B51
:108F600080021D68296800F0E7FA24686A6823789F
:108F7000002B00D16EE01C9D911CEB8849006B809A
:108F80002B892E1C2B800B1FEB181D887552991EE8
:108F90000988D9806178002903D0079D6FB27F00CE
:108FA00039E0023B013A39D35E88DD8803216156FE
:108FB0007519079E4D431F8871B21E89BE194E4315
:108FC0000221AD1961569E88714369188911414388
:108FD00009141981E5E7032565575988DE886D0076
:108FE000AC460D1CB14200D2351CADB266466E4394
:108FF0001D89B4461E88311CAE4200D2291C0225B0
:10900000655789B29E887943754361444D19AD1106
:1090100045432D141D81023B013ADCD2099F0D20EE
:109020007F68049720560622A15E0823E25E0C2387
:10903000E3560090381CFCF73FFF764B80021C681B
:10904000616800F079FA724B226819680B78002B7E
:109050000CD161E0531C1C9F5B00FB18013ADDD36F
:109060001988023B41430914D980F7E71B9CE38828
:10907000251C63802389261C2380941C6400231FE5
:10908000EB181D8835539C1E2488DC804C78002CFE
:1090900003D0079C67B27F003AE0023B013A00D25E
:1090A0003BE75E88DD8803240C577519079E6543EE
:1090B0001F8874B21E89BE1966430224AD190C576D
:1090C0009E8874432C19A411444324141C81E4E7A2
:1090D00003254D575C88DE886D00AC46251CB442E4
:1090E00000D2351CADB264466C431E881D89A4466F
:1090F000341CAE4200D22C1C02254D57A4B29E88CF
:109100007C43754364446519AD1145432D141D819D
:10911000023B013ADCD200E7531C1B9D5B00EB18BD
:10912000013A00D2F9E61988023B41430914D9807B
:10913000F6E7099E1027D95F7068002407948842DB
:109140000EDD12255A5F1B7D01265BB20093231CA6
:10915000FCF7B2FE10231B1A9B000B900D93079691
:109160002C4B002118682A4B07681B68BC460E93DD
:10917000099167464368791E00D299E01B9C4A001A
:10918000A2180F92013B00D290E0079D8468002D49
:1091900042D0664666430896F6180A9F0136760066
:1091A000BD5B5F1C2AB2D243D2172A408D1C654397
:1091B00002967D190A9E6D00AE5F12B2039696422A
:1091C00000DA0392089E341B3C190A9F6400E45F96
:1091D000944200DA141C039E0A9F3519029C3E1922
:1091E0000224375F141EBC4200DA3C1C023E2D19DB
:1091F0000027F45F161EA64200DA261CAD190B9C50
:109200000D9E65437243AA1892110CE0858E0000F2
:10921000440E0020D403002067467C431C1901340F
:109220000A9D6400625FC41DE47F002C05D1D60F47
:10923000642595427441644222400E9E3479002C8C
:1092400007D01C9F5C003C1924890F9D121B2C89A0
:10925000121B109EB24218DD069F0B243C579C4205
:1092600000DAFB72069D0A242C579C4200DDAB728B
:10927000069E092434578C4200DA7172069F082436
:109280003C578C4203DD397201E0002A04DD099C61
:10929000944202DA099200E00022846865466C4339
:1092A0001C1901340C9EA400A2516BE78C4660E7A8
:1092B0000999069C0022216012A98A8082680568AB
:1092C0000C9E4B708A707C2301325B429200CB7003
:1092D000B218832305200B710D70FCF733FD034892
:1092E0001199FBF7E5F815B0F0BDC046858E00007A
:1092F000014B18687047C046E003002000487047E3
:10930000A4070000014B18687047C046E003002026
:10931000024B1868F930FF307047C046E003002068
:10932000C4235B005843034B1B681818C3239B00DE
:10933000C0187047E00300200A235843034B1B6802
:109340001818BB239B00C0187047C046E0030020DC
:10935000014B18607047C046480E0020014B18684A
:109360007047C046480E002000487047B4B7000060
:1093700038B5F9F7B3FF0F4B41791B6801255960E8
:109380004279941C2A40A2189A6082791A604A4352
:10939000DA60427902219A61AA40DA610268596171
:1093A0001A62C2791A6101795A1DD177027906339E
:1093B000DA7738BDD403002010B5124C1249134A95
:1093C000206800F039F92068F9F782FF2068B4308E
:1093D000F7F70EFD2068EC30FCF7A2FD2068F430B2
:1093E000FDF754FB2068F530FF30FCF78BF9FFF7F1
:1093F000BFFF074C201CF9F783FF064BE018FCF772
:10940000A7FD10BDE003002010B00000A40700007D
:10941000B4B70000C503000038B5174BC424596821
:1094200064000A781B685443C2229200A4181C19D5
:10943000124B201D1860F9F757FFBA235B00E5189F
:10944000281CFFF727FD201CF830F7F7DDFC8621EC
:1094500049006018FCF770FD90225200A018FDF73B
:1094600021FB281CFCF75AF9054B9E341B68227817
:109470000733DA7738BDC046E0030020480E0020ED
:10948000D4030020014B5B6818707047E003002094
:10949000014B5B6818787047E0030020002934D046
:1094A0000123002210B488422CD301242407A142B6
:1094B00004D2814202D209011B01F8E7E400A14273
:1094C00004D2814202D249005B00F8E7884201D30E
:1094D000401A1A434C08A04202D3001B5C082243E6
:1094E0008C08A04202D3001B9C082243CC08A04257
:1094F00002D3001BDC082243002803D01B0901D043
:109500000909E3E7101C10BC7047002801D00020B7
:10951000C04307B4024802A14018029003BDC046F0
:10952000D90000000029F0D003B5FFF7B9FF0EBC49
:109530004243891A1847C046002941D010B4041C80
:109540004C40A44601230022002900D549420028AE
:1095500000D5404288422CD301242407A14204D2E2
:10956000814202D209011B01F8E7E400A14204D2C2
:10957000814202D249005B00F8E7884201D3401AD9
:109580001A434C08A04202D3001B5C0822438C08FB
:10959000A04202D3001B9C082243CC08A04202D365
:1095A000001BDC082243002803D01B0901D0090955
:1095B000E3E7101C6446002C00D5404210BC704705
:1095C000002806D003DB0020C043400801E08020D3
:1095D000000607B4024802A14018029003BDC0462D
:1095E000190000000029EBD003B5FFF7A7FF0EBC60
:1095F0004243891A1847C0467047C046F8B50D1C4B
:10960000041C081C111C161CFFF796FF311C071CBC
:10961000281CFFF7E7FF002D05DB002908DB27608A
:10962000201C6160F8BD0029F9DD013F8919F6E7CA
:109630000137891BF3E7C046F0B50F2A35D9031C63
:109640000B439C0735D1161C103E360935014519D0
:1096500010350C1C031C27681F6067685F60A768D3
:109660009F60E7681034DF601033AB42F3D1731CA6
:109670001B01C518C9180F231340032B1BD91C1F2E
:10968000A4080134A4000023CE58EE500433A342B2
:10969000FAD1ED18C91803231A4005D00023CC5C79
:1096A000EC5401339342FAD1F0BD051C002AF5D1E8
:1096B000FAE7051CF2E71A1CF8E7C046F0B5830785
:1096C00046D0541E002A42D0CEB2031C032503E02C
:1096D000621E002C3BD0141C01335A1E16702B4204
:1096E000F6D1032C2BD9FF250D402A0215432A045D
:1096F00015430F2C15D9271C103F3F091E1C3A019A
:109700001036B6181A1C156055609560D560103279
:10971000B242F8D101373F010F22DB191440032C6C
:109720000DD9271FBF08BA001E1DB6181A1C20C26B
:10973000B242FCD10137BF000322DB191440002CD8
:1097400005D01C19C9B219700133A342FBD1F0BD79
:10975000141C031CC5E7C046AE0174033B05020799
:10976000CD08940A590C1F0E0600000008000000E6
:10977000FF000001FF01FF0100FF0100FFFF0101E9
:1097800000010203040405060708090A0B0B0C0D6F
:109790000E0F101111121314151516171818191A87
:1097A0001B1B1C1D1D1E1F1F2021212223232424BF
:1097B0002525262727282829292A2A2B2B2C2C2D1A
:1097C0002D0000007804EF08660DDB115016C21A58
:1097D000331FA1230C28742CD93039359639EE3D2E
:1097E00042429046D94A1B4F58538E57BE5BE65FA4
:1097F00007641F68306C397038742F781C7CFF7FC9
:10980000D983A8876D8B278FD5927996109A9B9DC7
:109810001BA18DA4F3A74BAB97AED4B104B526B86A
:1098200039BB3EBE34C11BC4F2C6BAC973CC1BCF10
:10983000B3D13BD4B2D619D96EDBB3DDE6DF08E293
:1098400018E416E603E8DDE9A5EB5BEDFEEE8FF02C
:109850000DF277F3CFF414F646F764F86FF967FA70
:109860004BFB1BFCD8FC81FD17FE98FE06FF5FFF3B
:10987000A5FFD7FFF5FFFFFF00000E0022006300E9
:10988000000140002F001E0017001000B502390132
:109890007E00000048000020E803002000000000D7
:1098A000FF000000000000000000000000000000B9
:1098B00000000000000000000000000000000000A8
:1098C0000000000000000000000000000000000098
:1098D0000000000000000000000000000000000088
:1098E0000000000000000000000000000000000078
:1098F0000000000000000000000000000000000068
:109900000000000000000000000000000000000057
:109910000000000000000000020000000000000045
:109920000000000000000000000000000000000037
:109930000000000000000000000000000000000027
:109940000000000000000000000000000000000017
:109950000000000000000000000000000000000007
:1099600000000000000000000000000003000000F4
:1099700000000000000000000000000000000000E7
:1099800000000000000000000000000000000000D7
:1099900000000000300400203004002020040020DB
:1099A000500100200A00000000101C00010000000F
:1099B00000000000000000000000000000000000A7
:1099C0000000000000000000000000000000000097
:1099D0000000000000000000000000000000000087
:1099E0000000000000000000000000000000000077
:1099F0000000000000000000000000000000000067
:109A00000000000000000000000000000000000056
:109A10000000000000000000000000000000000046
:109A20000000000000000000000000000000000036
:109A30000000000000000000000000000000000026
:109A40000000000000000000000000000000000016
:109A50000000000000000000300400201C05002071
:109A60004D050020450500203D05002000000000B8
:109A7000C803002000000000C6030020B803002037
:109A8000AA030020A9030020000000001C050020FC
:109A9000CC0200202C05002002000000200E002037
:109AA0000000000000000000070000003B0500204F
:109AB000A50300203C05002000000000000000007D
:109AC0000000000000000000800300206C03002064
:109AD000000000000000000000000000580300200B
:109AE0000000000044030020000000002C030020C0
:109AF0000000000010030020000000000000000033
:109B000000000000F8020020E4020020D002002043
:109B1000A10300209C030020000000003705002066
:109B200000200060C802002034050020E002002070
:109B3000010000000400000058020020350500204C
:109B4000F40200200100000001000000BC0200201F
:109B50000B0300200803002003000000040506009A
:109B6000102000005C0200202503002020030020BC
:109B7000050000000401060104001020303100003F
:109B80002C0200203F0300203C03002003000000C3
:109B90000401060010200000B0030020360500205C
:109BA00054030020010000000400000024020020F3
:109BB0006A0300206803002002000000020E00106B
:109BC000480200207C030020540200200300000013
:109BD000001011000C0200209603002090030020CA
:109BE000060000001708080C0A08002030405070DA
:109BF00001000000000020050100200100FF0020FE
:109C000001000000B4030020006008010001000012
:109C10000000000000000000000005004D49500059
:109C200000000000000400006C05002094050020E6
:109C3000A40500205C06002058060020FFFFFFFF5F
:109C4000FFFFFFFFFFFFFFFFFFFFFFFFFFFFFFFF24
:109C5000FFFFFFFFFFFFFFFFFFFFFFFF3801500186
:109C60004D344850435554320000000000000601B6
:109C700070B50420FCF731F900F0DEFAFBF71AFFAB
:109C8000FCF71CFF4E4C4F4B4F4EA8300360326820
:109C900023684E485A604E4900F046FA23684D4DFD
:109CA0001A68291C01321A604B4800F03DFA2368FB
:109CB000291C1A68494801321A6000F035FA2368F5
:109CC000291C1A68464801321A6000F02DFA2368F0
:109CD00044481A68444901321A6000F025FA2368A2
:109CE00036681A68DE6001321A604048404900F068
:109CF0001BFA23683F489A683F4901329A6000F096
:109D000013FA23683D489A683D4901329A6000F091
:109D10000BFA23683B489A683B4901329A6000F08D
:109D200003FA236839489A68394901329A6000F089
:109D3000FBF9236837489A68374901329A6000F086
:109D4000F3F9236835489A68354901329A6000F082
:109D5000EBF9236833489A68334901329A6000F07E
:109D6000E3F9236831489A68314901329A6000F07A
:109D7000DBF923682F489A682F4901329A6000F076
:109D8000D3F923682D489A682D4901329A6000F072
:109D9000CBF923682B489A682B4901329A6000F06E
:109DA000C3F9236829499A68294801329A6000F06A
:109DB000BBF923689A6801329A60FCF77FFE70BD98
:109DC0004801002041A00000280E0020192C0000AE
:109DD000A9A10000B3A10000A52E0000355300008A
:109DE000E52F0000C1170000099E0000FD2B0000B8
:109DF000F59D000021110000119E000001100000DF
:109E0000219E0000858E0000079E00005D6C000012
:109E100025A00000911D0000A59E0000E517000090
:109E2000DD9E0000E12900000B9E0000B11E000035
:109E30000D9E0000B56200000F9E0000892E0000FC
:109E4000099F000009830000BD9F0000059E0000DF
:109E500069800000024B1B681A68596806C3704786
:109E6000D4030020704770477047704770477047B1
:109E700007B5002201AB1A800198FAF785FA07BDF1
:109E8000F8B5FCF709FE1C4B1C680023261CE06A91
:109E900074363278984204D1616B0123283100DB9B
:109EA000031CE76C13433370FB1E144D162B1AD89A
:109EB000A36B1D2B17DC632815DC216C0E2912DC2B
:109EC000FFF73AFB05280EDCE4342378002B0AD197
:109ED0000B4B1B685B691B78012B01D8052F02DD3A
:109EE0002B68013300E000232B602B681E2B01DD63
:109EF00001233370F8BDC046400000201C04002040
:109F00004400002038B5F6F791FF041CFCF7D6FD9D
:109F10006269051C13788635002B04D02B78002B42
:109F200001D1FCF747FF2B78002B06D061690B7835
:109F3000002B02D12069FCF70BFF38BD08B5FFF7F5
:109F4000D7F9F9F7C5F9FFF713FA064B1B6803CBEE
:109F5000F9F758FA0020FAF73BF8F9F79FFFF6F700
:109F60000DFF08BDD4030020F0B589B0F9F7B6F9AC
:109F70002649102204A8FFF75FFBFAF77BFA244B6F
:109F800024491A68244C13680E682768013B22D3C1
:109F900051680D1C5D436C186D00640089000395C9
:109FA000039D0439AC42F1D0F569023C02942C19AE
:109FB0000194BD69440000946C58009DA44610357E
:109FC0006C462D5B64462C1BA446019C2588654489
:109FD0002580029CE4E70F4F0F4B12693D681E6815
:109FE00053009200023B043A991C0DD02C6A376A48
:109FF000E118BC580F883F1B4400BC4610346F4624
:10A00000E45B64440C80EDE709B0F0BDF896000015
:10A01000D4030020440000204000002038B5F6F7AB
:10A02000FFFE041CFCF738FD201CF0300378002BE9
:10A0300023D0124B00221C681E23216BC968C95E05
:10A04000002900D10122023B991CF6D10C4B1B6860
:10A05000DD6A002D11D1596B00290ED1F433002A8D
:10A060000AD01A68FE2A01DC01321A601B68052B2F
:10A0700003DD0023037000E01A6038BD44000020B7
:10A080004000002008B5FBF76DFD012805D0034B0B
:10A090001B681869596900F0EBF808BD44000020FE
:10A0A00070B5041C0D1CFBF7EFFD002802D0012841
:10A0B0000CD035E01B4B6D001B681B691B69EA5A0D
:10A0C000FF23FE2A00D8D3B2637129E0154B690043
:10A0D0001B681A691269895AFF22FE2900D8CAB280
:10A0E00062711B69AD005969022349190325CB56DA
:10A0F0004D570126ED1A00238E57CB56F61AB5425E
:10A1000007DD281C0521FFF717FA4519A571E6712F
:10A1100006E0301C0521FFF70FFA8619A671E571DC
:10A1200070BDC0464400002038B5051C08200C1C3A
:10A13000FBF7D3FE0560446038BD70B52F4C304D41
:10A14000304E002810D02068AA796B79291C427102
:10A1500083712F310B30FFF76FFA2368291C181C0D
:10A160002F309A790B310FE020686A79AB79291C7E
:10A17000427183710B310B30FFF75EFA2368291CA3
:10A18000181C9A792F302F31FFF756FA226833685E
:10A190001079591DC87712790633DA772068F9F7F4
:10A1A00097F8226833685179012559605079841CE9
:10A1B00028402018986090790C1C44431860DC609B
:10A1C000547902259C616400DC6114685D611C6245
:10A1D000D2791A61F9F716F9F7F722FB0020F9F79F
:10A1E000F7FEF9F75BFEF6F7C9FD0020F8F720FA55
:10A1F000F9F780F8F8F754F870BDC0464C0100201C
:10A2000010B00000D403002008B50020FFF795FF30
:10A2100008BD08B50120FFF790FF08BD38B5041C44
:10A22000081C002A07D0D118584362434D1010185B
:10A230004019FFF781F938BD38B5FCF739FC041C2B
:10A24000B820FBF74AFE094DB82228600021FFF72D
:10A2500035FA231C52333C341B7820786421584350
:10A26000FFF76AF92D68B035286038BD4C0E002024
:10A27000F0B599B00E1C041CFCF71AFC0C90FCF70E
:10A280000BFC1190FBF770FE119B0122F0331B7841
:10A2900000259A40131C119AF13212789B1A119AD8
:10A2A000F23212789B1ADBB21593FCF707FCCC4B09
:10A2B0000F901B6810951393CA4B0B951B681B6A74
:10A2C0000A935B00023B9F1C0CD02769109DFA5A31
:10A2D000954200DA1092E7680B9DFA5E9542F1DA3A
:10A2E0000B92EFE70A9B0F9D11339B00EB1808932D
:10A2F0000A9F013F0A9700D2C2E00A9DE0686F0002
:10A30000C35F002B00D1B7E00C9B21690F9A523339
:10A310001B78C85B126A09930C9B90420ADD1B698B
:10A320000C9A0693191C0C9B14322833FBF7E0FDA2
:10A33000051C01E03D331D78F6F772FDF03003781F
:10A34000002B05D00C9B3E331B789D4200DA1D1C70
:10A350000C9B53331B78002B02D16420844649E0C8
:10A360009F4B09991B688C461A1CB43212921078C4
:10A37000149000281FD1E1686046C95F64220D91E6
:10A38000684351431A1CAC32814212DD0D99A94237
:10A390000FDC106801300990106011980999DA30CB
:10A3A0000078814207D1129901200870149810603A
:10A3B00001E000211160191CB4310D910A78002AC6
:10A3C00014D0E268D05F1A1CAC32A8420CDD1068D1
:10A3D0000C990130106041310978884206D10D99FD
:10A3E00000200870106001E000211160B4331B7878
:10A3F000002BB2D00F9A0A9813183433E2681B78F6
:10A40000D219002B05D00C995BB2413109788B42EF
:10A410001DDC0021535E642061464D435843216991
:10A42000A84211DB0C98CD5B4830AC460078109DFB
:10A4300068438011844507DB0C980B9DC06C059028
:10A4400068438011834217DA0023CB530EE066493C
:10A450000020135E4B430C993C3109784D43614613
:10A460004D43AB4208DA25690023EB53089F138064
:10A470003B602378013B2370089D043D089537E736
:10A4800000232370574B0F9D1B681A6A531EAA188E
:10A4900033320A920C225F005343139DEB180F9D39
:10A4A0001093333517950A9D0F9817992B1A343B43
:10A4B0000B938D4200D131E2E0680A9DC35F002B0F
:10A4C00000D1F0E12A780C9B0132D2B22A704133DC
:10A4D0001B7852B2991D8A4201DD04332B700A9811
:10A4E00000254557012D00DCC9E1A81C0321FFF719
:10A4F00079F873680991B268022D38D10F98D95F45
:10A500008069D25B0F9D049040109446EA690D1A51
:10A51000EB17ED185D40401B7F281BDC65462BB216
:10A520005210981AC51740196840121A7F2A11DC78
:10A530006268A568D05F401AE95FC91AFDF77CFC24
:10A540000B2807D970686168C35BB268CB53D35BD3
:10A55000A568EB530323013B11D36068109DC15BD9
:10A560005A00A068A952C15BAA18D180F3E7099DDF
:10A57000D95B6B00109DEB181980D25BDA800A98CA
:10A5800000254557032D00DC67E10999109A4B001F
:10A59000D3180893081C1B88043003210D93FFF780
:10A5A00021F810984900089B41180A88DB88C9885F
:10A5B00013929C4612916268042D17D17168D05F86
:10A5C000CB5FA568C31ADA17B1689B185340E85FE0
:10A5D000CA5F801AC2178018504018181EE0C04683
:10A5E0004C0E0020D403002010270000DA490B9DF8
:10A5F00009686B00CB18D05F1A1C82320025525FAD
:10A60000A568821AD01712189633E95F42400025D8
:10A61000585F081AC117401848401018CE4B62689E
:10A620000B991B68D55B4A009A18111C82310D806A
:10A63000A5689632E95B0B9D118059190A1C783286
:10A640001378002B06D0119BF8331B88984208DC46
:10A65000002305E0119BFA331B88984201DB01239C
:10A6600013700B1C78331B78002B38D1119A119B77
:10A67000F63212888021F4331B8800924A00FBF7DF
:10A680001BFC65680B90ED190020295E0995089D5B
:10A69000A2680020285ED5190B1ADA179B185340C0
:10A6A0000D930022AB5E9C46089B06229A5E634691
:10A6B0009A1AD317D2185A400D9B9A180D920D9BD7
:10A6C0000B9AFFF7ABFD0999089A08800620105EE7
:10A6D0000023E95E0B9A0D9BFFF7A0FD96E00D9D10
:10A6E000624628B2139D11B22BB2C31ADA0FD318E7
:10A6F000129A5B1015B24D1B0E93EB0F5D196D1086
:10A7000012956568ED1916950022AD5E0D95A56848
:10A71000ED1913950022AD5E14950E9D2B180D9D1D
:10A72000EB1A129DD8176918149D1B18691A43401B
:10A73000C8170918414000255B180B95802B01DDD7
:10A74000803B0B93099803210530FEF74BFF109DCA
:10A75000119B49006918089D0291F1331B7806216D
:10A76000695E159D09934D43119B0298F2331B7846
:10A770000621415EAC46099D039314986943039DED
:10A78000119B4543F0331B788C44119A65441D415D
:10A79000F3321278AC46129D0B985543291C19418F
:10A7A000614414918021C9004518089968101290DD
:10A7B0000020095E15984843844602980021415EB6
:10A7C0000998414303988C440D9948430E9960447D
:10A7D0004A4318411A4180180B990D9A129B514314
:10A7E00080024018C018291CFEF7A6FE16990880A2
:10A7F000149A139993020020085E0B9A291C504367
:10A800001818129BC018FEF797FE139D2880E56864
:10A81000F168ED19C85F09950022A95E0C9D083505
:10A8200008953E23EA5E431ADD175B196B40FFF77C
:10A83000F5FC099D316928802569C85BED192988D7
:10A840000995089D431A3E22AA5EDD175B196B40ED
:10A85000FFF7E4FC099D288011E060687568C31962
:10A860000022995EEA5FA0688A185210B5681A80C3
:10A87000C3190022995EEA5F8A1852101A800C9B55
:10A880000A9D00224133AA561B789A4204DC012318
:10A89000E0685B42C35302E02378013323700A9DD2
:10A8A0000023AB7232E00C9A0021413269561278D3
:10A8B000914223DDF068C25F002A27D0AA7A0C9962
:10A8C0000132D2B2AA724231097852B28A4201DD13
:10A8D0002B701BE071686268CB5BB568D353EB5B90
:10A8E000A068F168C353CB5BE2683569D353EB5B77
:10A8F0002069C35323780133237007E00A9D164A69
:10A900002B7012680B9D5219783213700A9D023F0A
:10A91000013D0A95109D0C3D1095C4E5031C7A334A
:10A9200000221A700D4B1B681D6944193B356D00E0
:10A9300045199130913404350890089FBC4260D08D
:10A940002B88002B13D00C27EA5F1BB2002A07DCF0
:10A950000C9A3F3206E0C0464C0E0020D403002083
:10A960000C9A40321278934201DA00232B80298816
:10A97000002927D023787F2B01D0013323700026B4
:10A98000A657022E0DDD0C9B0C22A85E09B20833DF
:10A990003E27DA5F431ADF17DB197B40FFF73EFCE7
:10A9A00028800C9B43331B789E4203DC01235B42CF
:10A9B0002B8004E00F9B7A331A7801321A7000233F
:10A9C00063711BE00C9B00224333A2561B789A4212
:10A9D00013DDAB89002B11D062790C980132D2B211
:10A9E00062714430007852B2824206DC2B800F9BA9
:10A9F0007A331A7801321A7000E02170013C023D6E
:10AA00009BE719B0F0BDC046FFFFFFFFFFFFFFFF50
:10AA1000FFFFFFFFFFFFFFFFFFFFFFFFFFFFFFFF46
:10AA2000FFFFFFFFFFFFFFFFFFFFFFFFFFFFFFFF36
:10AA3000FFFFFFFFFFFFFFFFFFFFFFFFFFFFFFFF26
:10AA4000FFFFFFFFFFFFFFFFFFFFFFFFFFFFFFFF16
:10B05000FFFFFFFFFFFFFFFFFFFFFFFF50010601A4
:10B060004D344850504154320000000000000601A9
:10B070000A000000011C1000010000020304050684
:10B080000708090A0B0C0D0E0F1011122728292A88
:10B090002B2C2D2E2F30310000000000000000145A
:10B0A00015161718191A1B1C1D1E1F2021222300FC
:10B0B0000000000000000000000000000000000090
:10B0C000000000000000000000000000003718052C
:10B0D00000BF000F000000000000000000000000A2
:10B0E0000000000000000000000000000000000060
:10B0F00000000000000000F0000000000000000060
:10B10000000000000000000000000000000000003F
:10B1100000000000830000000001E1A10800000918
:10B120000303000053355F4E454F00000000000050
:10B13000000000000A6E6E000100FFFFFFFFFFFF2E
:10B14000FFFFFFFF0A052C01F401A000C800640006
:10B150000005641E1E0A0305100F3C000A0A3C008D
:10B160000080000038040000800700000A00000092
:10B17000E803000000000000C003000064000000BD
:10B1800001000000010000000100000001000000BB
:10B1900005000000000040008000C400FF005F00C8
:10B1A0005F005F005F005F005F005F005F005F00A7
:10B1B0005F005F005F005F005F005F005F005F0097
:10B1C0005F005F005F000000000000000000000062
:10B1D000000000000000000000000000000000006F
:10B1E000000000000000000000000000000000005F
:10B1F000000000000000000000000000000000004F
:10B2000002000000000040008000C400FF00800039
:10B2100080000000000000008000800000000000AE
:10B22000000080008000000000000000800080001E
:10B23000000000000000000000007A0268043C00EA
:10B24000C8001E00B0045E01F401010020035A0092
:10B25000230018010613133D800200012D00780021
:10B260002C0100000100000000BF000F00000000E2
:10B2700000000000000000000000000000000000CE
:10B28000000000000000000000000000000000F0CE
:10B2900000000000000000000000000000000000AE
:10B2A000000000000000000000000000001E000F71
:10B2B000000000000000000000000000000000008E
:10B2C000000000000000000000000000000000007E
:10B2D000000000F00000000000000000000000007E
:10B2E000000000000000000000000000000000005E
:10B2F000800000004003331CD10000710A48F61C96
:10B300000000003718053718003718050000000046
:10B31000000000000000000000000000000000002D
:10B32000000000000000000000000000000000001D
:10B33000000000000000000000000000000000000D
:10B3400000000000000000000000000000000000FD
:10B350000000000000000000000000000000FFFFEF
:10B360000A14380703000000FFFF0A14380703001F
:10B370000000FFFF0A1438070300000000BF000FA1
:10B3800000000000000000000000000000000000BD
:10B3900000000000000000000000000000000000AD
:10B3A000000000F0000000000000000000000000AD
:10B3B000000000000000000000000000000000008D
:10B3C000009E000F000000000000000000000000D0
:10B3D000000000000000000000000000000000006D
:10B3E00000000000000000F000000000000000006D
:10B3F000000000000000000000000000000000004D
:10B4000000000000800000004003331CD1000071E8
:10B410000A48F61C000000371805371800371805D1
:10B42000000000000000000000000000000000001C
:10B43000000000000000000000000000000000000C
:10B4400000000000000000000000000000000000FC
:10B4500000000000000000000000000000000000EC
:10B4600000000000000000000000000000000000DC
:10B47000641E96005000000007000000FF7F00805F
:10B48000FF7F00800103000000005A0308000080D5
:10B4900007070F090CF44000E8028A025E019600DB
:10B4A0003000000064000000060000000B001300E4
:10B4B00023003E0050005A00000000000000000081
:10B4C0002D004600960096009600960000000000B1
:10B4D000000000004B28A01E0F0201020200000025
:10B4E00001000000010000000101010001000A0D3F
:10B4F000010028005A000A3C0A3C01002C01E80324
:10B500001000000000BF000F00000000000000005D
:10B51000000000000000000000000000000000002B
:10B520000000000000000000000000F0000000002B
:10B53000000000000000000000000000000000000B
:10B540000000000000000000009E000F000000004E
:10B5500000000000000000000000000000000000EB
:10B56000000000000000000000000000000000F0EB
:10B5700000000000000000000000000000000000CB
:10B58000000000000000000000000000800000003B
:10B590004003331CD10000710A48F61C000000373C
:10B5A00018053718003718050000000000000000DB
:10B5B000000000000000000000000000000000008B
:10B5C000000000000000000000000000000000007B
:10B5D000000000000000000000000000000000006B
:10B5E000000000000000000000000000000000005B
:10B5F0000000000000000000641E8C0050000000ED
:10B6000007000000FF7F0080FF7F00800103000033
:10B6100000005A030800008007070F090CF44000DF
:10B6200084022602FA0032003000000064000000AC
:10B63000060000002800320037004600600071005C
:10B64000000000000000000019003C005A00A000AB
:10B650000401540100000000000000004B19A01E6E
:10B660000F020102020000000100000001000000C2
:10B670000101010001000A0D010028005A001446D2
:10B68000144601002C01E8031000000000BF000F69
:10B6900000000000000000000000000000000000AA
:10B6A000000000000000000000000000000000009A
:10B6B000000000F00000000000000000000000009A
:10B6C000000000000000000000000000000000007A
:10B6D000009E000F000000000000000000000000BD
:10B6E000000000000000000000000000000000005A
:10B6F00000000000000000F000000000000000005A
:10B700000000000000000000000000000000000039
:10B7100000000000400000004003331CD100007115
:10B720000A48F61C0000013710041004003710040A
:10B730000000000000000000000000000000000009
:10B7400000000000000000000000000000000000F9
:10B7500000000000000000000000000000000000E9
:10B7600000000000000000000000000000000000D9
:10B7700000000000000000000000000000000000C9
:10B78000641EAA005000000007000000FF7F008038
:10B79000FF7F00800103000000005A0308000080C2
:10B7A000070701090CF44000E8028A025E019600D6
:10B7B0003000000064000000060000002800320095
:10B7C000370046006000710000000000000000002B
:10B7D00019003C005A00A0000401540100000000C0
:10B7E000000000004B19A01E0F0201020200000021
:10B7F00001000000010000000101010000000A0D2D
:10B80000010028005A002D5F010101002C01E8030E
:10B8100010000000060707080809090A0A0A0B0CAD
:10B820000C0C0D0D0D0D0D0D0D0E0D0E0D0D0D0E47
:10B83000060707080808090A0A0A0B0A0B0C0C0D70
:10B840000D0D0D0D0D0D0D0D0D0D0D0D0606070742
:10B8500008080909090A0B0B0B0C0C0C0C0C0C0D3D
:10B860000C0D0C0C0C0C0C0D06060707080809093A
:10B87000090A0B0B0B0B0C0C0C0C0C0C0D0D0D0C0E
:10B880000C0C0D0D06060707070809090909090B25
:10B890000C0B0C0C0C0C0C0C0C0D0C0C0C0C0C0DE7
:10B8A00006060607070808090909090A0B0B0C0C0C
:10B8B0000C0C0C0C0C0C0C0C0C0C0C0C05060607E0
:10B8C0000708080809090A0A0B0B0B0B0B0B0B0DD9
:10B8D0000B0D0C0D0B0D0B0D0506060607070808D2
:10B8E000080909090B0B0B0B0B0B0B0C0B0C0B0CAE
:10B8F0000B0C0B0C050506060707070808080909C5
:10B900000A0B0A0B0B0B0C0B0B0B0B0B0B0B0B0B88
:10B910000505050606070708080809090A0A0A0BAB
:10B920000B0B0B0B0B0B0B0B0B0B0B0B040505067F
:10B93000060607070708090809090A0B0A0A0A0B7D
:10B940000B0B0A0B0B0B0B0B040505050606070773
:10B950000708080809080A0A0A0A0A0B0A0B0A0A51
:10B960000A0A0A0B04040505060607070707080864
:10B970000909090A0A0A0A0A0A0A0A0A0A0A0A0B29
:10B98000040405050606060707070808080909094B
:10B990000A0A0A0A0A0A0A0A0A0A0A0A040404051E
:10B9A0000505060607070707080809090A0A0A0A1B
:10B9B0000A0A0A0A0A0A0A0A040404050505060610
:10B9C00006070707070809090909090A0A0A090AEF
:10B9D000090A0A0A00000000000000000000000040
:10B9E0000000000000000000000000000000000057
:10B9F0000000000000000000000000000000000047
:10BA00000000000000000000000000000000000036
:10BA10000000000000000000000000000000000026
:10BA20000000000000000000000000000000000016
:10BA30000000000000000000000000000000000006
:10BA400000000000000000000000000000000000F6
:10BA500000000000000000000000000000000000E6
:10BA600000000000000000000000000000000000D6
:10BA700000000000000000000000000000000000C6
:10BA800000000000000000000000000000000000B6
:10BA900000000000000000000000000000000000A6
:10BAA0000000000000000000000000000000000096
:10BAB0000000000000000000000000000000000086
:10BAC0000000000000000000000000000000000076
:10BAD0000000000000000000000000000000000066
:10BAE0000000000000000000000000000000000056
:10BAF0000000000000000000000000000000000046
:10BB00000000000000000000000000000000000035
:10BB10000000000000000000000000000000000025
:10BB20000000000000000000000000000000000015
:10BB30000000000000000000000000000000000005
:10BB400000000000000000000000000000000000F5
:10BB500000000000000000000000000000000000E5
:10BB600000000000000000000000000000000000D5
:10BB700000000000000000000000000000000000C5
:10BB800000000000000000000000000000000000B5
:10BB900000000000000000000000000000000000A5
:10BBA0000000000000000000000000000000000095
:10BBB0000000000000000000000000000000000085
:10BBC0000000000000000000000000000000000075
:10BBD0000000000000000000001D1C1C1E2023238C
:10BBE0002527292B2C2E2E3031313233363A393756
:10BBF0003C3635343C1918191A1B1D1E20222324EB
:10BC0000252727292A2A2A2B2F3031302F2E2E2D77
:10BC100034191718191B1D1D1F202224242725261F
:10BC2000292B292B2D2E2F2E2E2D2D2C3119171887
:10BC3000191B1C1D2020212323272527292B292AD6
:10BC40002D2E2F2E2E2E2C2B30181718191B1C1DA5
:10BC50001F20212324252526292B292B2E2F2E2D6D
:10BC60002F2D2D2B31181718191B1C1D1F1F2123B9
:10BC700024252528282B292B2D302D2D2E2E2F291C
:10BC80002F191718191A1C1D1E21212324242527BA
:10BC9000282A282B2D2E2D2D2F2C2E292F18171723
:10BCA000191A1D1D1E202122242425272828282A70
:10BCB0002B2F2D2F2D2D2B2A2F181718191A1D1C3D
:10BCC0001D1F2122232325272829292A2B2D2C2D0E
:10BCD0002E2C2A292E18161718191B1C1D1E21215F
:10BCE000232325262728282A2B2C2B2B2B2B2929CD
:10BCF0002D17161617191A1B1E1F20212223242860
:10BD00002726282B2C2D2A2C2C2B29292D171616CB
:10BD100017191A1B1C1D20212223232B2726272B12
:10BD20002B2C2B2C2D2B28292C1716161819191BE8
:10BD30001C1D1F2122232326262728292B2B2A2BB3
:10BD40002C2B28292C16161717191B1B1D1E2022F9
:10BD500022232425272628292A2B2A2B2B2B292866
:10BD60002B16151617191A1C1D1E202223232426F4
:10BD70002827272A2B2B2A2D2C2B28292B1818195A
:10BD80001B1C1E1F2223252628282A2C2E2D2D3150
:10BD90003332323433332E2E2E00000000000000E8
:10BDA0000000000000000000000000000000000093
:10BDB0000000000000000000000000000000000083
:10BDC0000000000000000000000000000000000073
:10BDD0000000000000000000000000000000000063
:10BDE0000000000000000000000000000000000053
:10BDF0000000000000000000000000000000000043
:10BE00000000000000000000000000000000000032
:10BE10000000000000000000000000000000000022
:10BE20000000000000000000000000000000000012
:10BE30000000000000000000000000000000000002
:10BE400000000000000000000000000000000000F2
:10BE500000000000000000000000000000000000E2
:10BE600000000000000000000000000000000000D2
:10BE700000000000000000000000000000000000C2
:10BE800000000000000000000000000000000000B2
:10BE900000000000000000000000000000000000A2
:10BEA0000000000000000000000000000000000092
:10BEB0000000000000000000000000000000000082
:10BEC0000000000000000000000000000000000072
:10BED0000000000000000000000000000000000062
:10BEE0000000000000000000000000000000000052
:10BEF0000000000000000000000000000000000042
:10BF00000000000000000000000000000000000031
:10BF10000000000000000000000000000000000021
:10BF20000000000000000000000000000000000011
:10BF30000000000000000000000000000000000001
:10BF400000000000000000000000000000000000F1
:10BF500000000000000000000000000000000000E1
:10BF600000000000000000000000000000000000D1
:10BF700000000000000000000000000000000000C1
:10BF800000000000000000000000000000000000B1
:10BF90000000000000000000000000000000FFFFA3
:10BFA000FFFFFFFFFFFFFFFFFFFFFFFFFFFFFFFFA1
:10BFB000FFFFFFFFFFFFFFFFFFFFFFFFFFFFFFFF91
:10BFC000FFFFFFFFFFFFFFFFFFFFFFFFFFFFFFFF81
:10BFD000FFFFFFFFFFFFFFFFFFFFFFFFFFFFFFFF71
:10BFE000FFFFFFFFFFFFFFFFFFFFFFFFFFFFFFFF61
:10BFF000FFFFFFFFFFFFFFFFFFFFFFFFFFFFFFFF51
:10C00000FFFFFFFFFFFFFFFFFFFFFFFFFFFFFFFF40
:10C01000FFFFFFFFFFFFFFFFFFFFFFFFFFFFFFFF30
:10C02000FFFFFFFFFFFFFFFFFFFFFFFFFFFFFFFF20
:10C03000FFFFFFFFFFFFFFFFFFFFFFFFFFFFFFFF10
:10C04000FFFFFFFFFFFFFFFFFFFFFFFFFFFFFF22DD
:10C0500022061520FA6A875532A600005001060113
:00000001FF
